 AsiBlCfg64

 Timestamp is 57b35ea3 (Tue Aug 16 14:42:43 2016)

 Preferred load address is 0000000180000000

 Start         Length     Name                   Class
 0001:00000000 00005180H .text$mn                CODE
 0001:00005180 0000009bH .text$x                 CODE
 0002:00000000 000003d8H .idata$5                DATA
 0002:000003d8 00000008H .CRT$XCA                DATA
 0002:000003e0 00000008H .CRT$XCZ                DATA
 0002:000003e8 00000008H .CRT$XIA                DATA
 0002:000003f0 00000008H .CRT$XIAA               DATA
 0002:000003f8 00000008H .CRT$XIC                DATA
 0002:00000400 00000008H .CRT$XIZ                DATA
 0002:00000410 00000dd0H .rdata                  DATA
 0002:000011e0 00000008H .rtc$IAA                DATA
 0002:000011e8 00000008H .rtc$IZZ                DATA
 0002:000011f0 00000008H .rtc$TAA                DATA
 0002:000011f8 00000008H .rtc$TZZ                DATA
 0002:00001200 000008c0H .xdata                  DATA
 0002:00001ac0 000000bfH .edata                  DATA
 0002:00001b80 000000a0H .idata$2                DATA
 0002:00001c20 00000014H .idata$3                DATA
 0002:00001c38 000003d8H .idata$4                DATA
 0002:00002010 000008b2H .idata$6                DATA
 0003:00000000 0000071cH .data                   DATA
 0003:00000720 000006d8H .bss                    DATA
 0004:00000000 000005f4H .pdata                  DATA
 0005:00000000 000002c8H .rsrc$01                DATA
 0005:000002d0 0002cb90H .rsrc$02                DATA

  Address         Publics by Value              Rva+Base               Lib:Object

 0000:00000000       ___safe_se_handler_count   0000000000000000     <absolute>
 0000:00000000       __guard_fids_table         0000000000000000     <absolute>
 0000:00000000       ___safe_se_handler_table   0000000000000000     <absolute>
 0000:00000000       __guard_flags              0000000000000000     <absolute>
 0000:00000000       __guard_fids_count         0000000000000000     <absolute>
 0000:00000000       __ImageBase                0000000180000000     <linker-defined>
 0001:00000000       ?AddList@ControlPanelRegistration@@AEAA_NPEAUkey_path_entry@@PEAUreg_list_entry@@@Z 0000000180001000 f   CtrlPnlReg.obj
 0001:000001a0       ?RemoveList@ControlPanelRegistration@@AEAA_NPEAUkey_path_entry@@PEAUreg_list_entry@@@Z 00000001800011a0 f   CtrlPnlReg.obj
 0001:000002e0       ?FindValueName@ControlPanelRegistration@@AEAA_NPEAUHKEY__@@PEB_WPEA_WH@Z 00000001800012e0 f   CtrlPnlReg.obj
 0001:000003c0       ?IsRegistered@ControlPanelRegistration@@QEAA?AW4CPRegState@@XZ 00000001800013c0 f   CtrlPnlReg.obj
 0001:00000550       ?Register@ControlPanelRegistration@@QEAA_NXZ 0000000180001550 f   CtrlPnlReg.obj
 0001:00000680       ?UnRegister@ControlPanelRegistration@@QEAA_NXZ 0000000180001680 f   CtrlPnlReg.obj
 0001:000007b0       ?Show@ControlPanelRegistration@@QEAA_N_N@Z 00000001800017b0 f   CtrlPnlReg.obj
 0001:000009d0       ?SetChannel@BluLinkChannelControl@@QEAAXH@Z 00000001800019d0 f i AdapterInfo.obj
 0001:00000ac0       ?GetColor@BluLinkChannelControl@@QEAAKXZ 0000000180001ac0 f i AdapterInfo.obj
 0001:00000b00       ?SetChannelsPerDevice@DialogParameters@@QEAAXH@Z 0000000180001b00 f i AdapterInfo.obj
 0001:00000b70       ?AllocateBlulinkControls@DialogParameters@@QEAAXXZ 0000000180001b70 f i AdapterInfo.obj
 0001:00000d30       ?FoundAsiRegistryKey@AsiBluLinkConfigPerAdapterInfo@@QEAAHPEAVDialogParameters@@PEAUHKEY__@@@Z 0000000180001d30 f   AdapterInfo.obj
 0001:00000db0       ?GetChannelFromHpiControl@@YAHII@Z 0000000180001db0 f   AdapterInfo.obj
 0001:00000ec0       ?InitChannels@AsiBluLinkConfigPerAdapterInfo@@QEAAXPEAVDialogParameters@@PEAX@Z 0000000180001ec0 f   AdapterInfo.obj
 0001:00001210       ?SaveChannelToHpiControl@@YAXIIH@Z 0000000180002210 f   AdapterInfo.obj
 0001:000013e0       ?SaveChannels@AsiBluLinkConfigPerAdapterInfo@@QEAAXPEAVDialogParameters@@PEAX@Z 00000001800023e0 f   AdapterInfo.obj
 0001:000015f0       ?FoundAsiRegistryKey@AsiBluLinkConfigAdapterInfo@@AEAAHPEAVDialogParameters@@PEAUHKEY__@@@Z 00000001800025f0 f   AdapterInfo.obj
 0001:000016a0       ?InitChannelsPerDevice@AsiBluLinkConfigAdapterInfo@@AEAAXPEAVDialogParameters@@PEAUHWND__@@@Z 00000001800026a0 f   AdapterInfo.obj
 0001:000018c0       ?InitAdapterInfo@AsiBluLinkConfigAdapterInfo@@QEAAHPEAVDialogParameters@@PEAUHWND__@@_N@Z 00000001800028c0 f   AdapterInfo.obj
 0001:00001de0       ?SaveAdapterInfo@AsiBluLinkConfigAdapterInfo@@QEAAXPEAVDialogParameters@@_N@Z 0000000180002de0 f   AdapterInfo.obj
 0001:00001fc0       DllMain                    0000000180002fc0 f   BluLinkCfg.obj
 0001:00001ff0       ?ShowControlPanel_RunDll@@YAXPEAUHWND__@@PEAUHINSTANCE__@@PEADH@Z 0000000180002ff0 f   BluLinkCfg.obj
 0001:00002190       ?RegisterControlPanelApplet_RunDll@@YAXPEAUHWND__@@PEAUHINSTANCE__@@PEADH@Z 0000000180003190 f   BluLinkCfg.obj
 0001:00002320       ?DllRegisterServer@@YAJXZ  0000000180003320 f   BluLinkCfg.obj
 0001:00002470       ?DllUnregisterServer@@YAJXZ 0000000180003470 f   BluLinkCfg.obj
 0001:00002500       ?SetConflict@BluLinkChannelControl@@QEAAXPEAV1@@Z 0000000180003500 f i ChanControl.obj
 0001:00002580       ?ReplaceBackgroundColor@@YAXPEAUHWND__@@K@Z 0000000180003580 f   ChanControl.obj
 0001:000026b0       ?BluLinkChannelEditSubclassProc@@YA_JPEAUHWND__@@I_K_J11@Z 00000001800036b0 f   ChanControl.obj
 0001:00002810       ??1DialogParameters@@QEAA@XZ 0000000180003810 f i ConfigDialog.obj
 0001:00002870       ??1AsiBluLinkConfigAdapterInfo@@QEAA@XZ 0000000180003870 f i ConfigDialog.obj
 0001:00002900       ?KeyboardProc@KeyboardHook@@CA_JH_K_J@Z 0000000180003900 f   ConfigDialog.obj
 0001:00002990       ?CheckInitialSettings@DialogParameters@@QEAAXPEAUHWND__@@@Z 0000000180003990 f   ConfigDialog.obj
 0001:00002ba0       ?CreateGroupOfControls@DialogParameters@@QEAAPEAGPEAGHHKKK@Z 0000000180003ba0 f   ConfigDialog.obj
 0001:00002d10       ?CustomizeDialog@DialogParameters@@QEAAPEAEPEAEH@Z 0000000180003d10 f   ConfigDialog.obj
 0001:00003050       ?CheckTxConflicts@DialogParameters@@QEAAXPEAVBluLinkChannelControl@@@Z 0000000180004050 f   ConfigDialog.obj
 0001:000031a0       ?RunRebootDialog@DialogParameters@@QEAAHPEAUHWND__@@@Z 00000001800041a0 f   ConfigDialog.obj
 0001:00003290       ?CheckSampleRateMismatch@DialogParameters@@QEAAHPEAUHWND__@@@Z 0000000180004290 f   ConfigDialog.obj
 0001:00003430       ?GuiSamplerateChange@DialogParameters@@QEAAXPEAUHWND__@@H@Z 0000000180004430 f   ConfigDialog.obj
 0001:000035f0       ??0AsiScrollbar@@QEAA@PEAUHWND__@@HHH@Z 00000001800045f0 f i ConfigDialog.obj
 0001:00003690       ?HandleScrollMessage@AsiScrollbar@@QEAAXGG@Z 0000000180004690 f i ConfigDialog.obj
 0001:000037e0       ?InitControls@@YAXPEAUHWND__@@PEAVDialogParameters@@@Z 00000001800047e0 f   ConfigDialog.obj
 0001:00003df0       ?CalculateMaxScroll@@YAHPEAUHWND__@@@Z 0000000180004df0 f   ConfigDialog.obj
 0001:00003e80       ?SetChannelValue@@YAXPEAUHWND__@@PEAVBluLinkChannelControl@@PEAVDialogParameters@@_KH@Z 0000000180004e80 f   ConfigDialog.obj
 0001:00003f20       ?EditControlMessage@@YA_JPEAUHWND__@@_K_JPEAVDialogParameters@@@Z 0000000180004f20 f   ConfigDialog.obj
 0001:00004090       ?GetShutdownPrivilege@@YAXXZ 0000000180005090 f   ConfigDialog.obj
 0001:00004120       ?DialogProc@@YA_JPEAUHWND__@@I_K_J@Z 0000000180005120 f   ConfigDialog.obj
 0001:00004490       ?SetControlToBold@@YAXPEAUHWND__@@H@Z 0000000180005490 f   ConfigDialog.obj
 0001:00004580       ?RebootDialogProc@@YA_JPEAUHWND__@@I_K_J@Z 0000000180005580 f   ConfigDialog.obj
 0001:00004630       ?RunDialog@@YAXPEAUHWND__@@_N@Z 0000000180005630 f   ConfigDialog.obj
 0001:00004820       __security_check_cookie    0000000180005820 f   MSVCRT:amdsecgs.obj
 0001:000048a0       _CRT_INIT                  00000001800058a0 f   MSVCRT:crtdll.obj
 0001:00004aec       _DllMainCRTStartup         0000000180005aec f   MSVCRT:crtdll.obj
 0001:00004c64       __raise_securityfailure    0000000180005c64 f   MSVCRT:gs_report.obj
 0001:00004cb0       __report_gsfailure         0000000180005cb0 f   MSVCRT:gs_report.obj
 0001:00004d82       __CppXcptFilter            0000000180005d82 f   MSVCRT:MSVCR120.dll
 0001:00004d88       _amsg_exit                 0000000180005d88 f   MSVCRT:MSVCR120.dll
 0001:00004d90       _FindPESection             0000000180005d90 f   MSVCRT:pesect.obj
 0001:00004de0       _IsNonwritableInCurrentImage 0000000180005de0 f   MSVCRT:pesect.obj
 0001:00004e30       _ValidateImageBase         0000000180005e30 f   MSVCRT:pesect.obj
 0001:00004e60       __atonexitinit             0000000180005e60 f   MSVCRT:atonexit.obj
 0001:00004eb0       _onexit                    0000000180005eb0 f   MSVCRT:atonexit.obj
 0001:00004f60       atexit                     0000000180005f60 f   MSVCRT:atonexit.obj
 0001:00004f78       __security_init_cookie     0000000180005f78 f   MSVCRT:gs_support.obj
 0001:00005024       _RTC_Initialize            0000000180006024 f   MSVCRT:initsect.obj
 0001:0000505c       _RTC_Terminate             000000018000605c f   MSVCRT:initsect.obj
 0001:00005094       _initterm                  0000000180006094 f   MSVCRT:MSVCR120.dll
 0001:0000509a       _initterm_e                000000018000609a f   MSVCRT:MSVCR120.dll
 0001:000050a0       __clean_type_info_names    00000001800060a0 f   MSVCRT:tncleanup.obj
 0001:000050ac       __C_specific_handler       00000001800060ac f   MSVCRT:MSVCR120.dll
 0001:000050b2       __crt_debugger_hook        00000001800060b2 f   MSVCRT:MSVCR120.dll
 0001:000050b8       __crtUnhandledException    00000001800060b8 f   MSVCRT:MSVCR120.dll
 0001:000050be       __crtTerminateProcess      00000001800060be f   MSVCRT:MSVCR120.dll
 0001:000050c4       __crtCapturePreviousContext 00000001800060c4 f   MSVCRT:MSVCR120.dll
 0001:000050ca       _lock                      00000001800060ca f   MSVCRT:MSVCR120.dll
 0001:000050d0       _unlock                    00000001800060d0 f   MSVCRT:MSVCR120.dll
 0001:000050d6       __dllonexit                00000001800060d6 f   MSVCRT:MSVCR120.dll
 0001:000050dc       __clean_type_info_names_internal 00000001800060dc f   MSVCRT:MSVCR120.dll
 0001:000050e2       IsProcessorFeaturePresent  00000001800060e2 f   kernel32:KERNEL32.dll
 0001:000050e8       __CxxFrameHandler3         00000001800060e8 f   MSVCRT:MSVCR120.dll
 0001:000050f0       __GSHandlerCheck           00000001800060f0 f   MSVCRT:gshandler.obj
 0001:00005110       __GSHandlerCheckCommon     0000000180006110 f   MSVCRT:gshandler.obj
 0001:00005174       memcpy                     0000000180006174 f   MSVCRT:MSVCR120.dll
 0001:0000517a       memset                     000000018000617a f   MSVCRT:MSVCR120.dll
 0002:00000000       __imp_RegOpenKeyExW        0000000180007000     advapi32:ADVAPI32.dll
 0002:00000008       __imp_AdjustTokenPrivileges 0000000180007008     advapi32:ADVAPI32.dll
 0002:00000010       __imp_LookupPrivilegeValueW 0000000180007010     advapi32:ADVAPI32.dll
 0002:00000018       __imp_RegEnumValueW        0000000180007018     advapi32:ADVAPI32.dll
 0002:00000020       __imp_RegDeleteValueW      0000000180007020     advapi32:ADVAPI32.dll
 0002:00000028       __imp_RegDeleteKeyW        0000000180007028     advapi32:ADVAPI32.dll
 0002:00000030       __imp_RegQueryValueExW     0000000180007030     advapi32:ADVAPI32.dll
 0002:00000038       __imp_RegCreateKeyExW      0000000180007038     advapi32:ADVAPI32.dll
 0002:00000040       __imp_OpenProcessToken     0000000180007040     advapi32:ADVAPI32.dll
 0002:00000048       __imp_RegSetValueExW       0000000180007048     advapi32:ADVAPI32.dll
 0002:00000050       __imp_RegCloseKey          0000000180007050     advapi32:ADVAPI32.dll
 0002:00000058       \177ADVAPI32_NULL_THUNK_DATA 0000000180007058     advapi32:ADVAPI32.dll
 0002:00000060       __imp_HPI_Object_GetValueEntity 0000000180007060     asihpi64:ASIHPI64.dll
 0002:00000068       __imp_HPI_Entity_Unpack    0000000180007068     asihpi64:ASIHPI64.dll
 0002:00000070       __imp_HPI_Entity_Free      0000000180007070     asihpi64:ASIHPI64.dll
 0002:00000078       __imp_HPI_AdapterGetProperty 0000000180007078     asihpi64:ASIHPI64.dll
 0002:00000080       __imp_HPI_Object_GetInfo   0000000180007080     asihpi64:ASIHPI64.dll
 0002:00000088       __imp_HPI_Entity_AllocAndPack 0000000180007088     asihpi64:ASIHPI64.dll
 0002:00000090       __imp_HPI_Universal_Set    0000000180007090     asihpi64:ASIHPI64.dll
 0002:00000098       __imp_HPI_SubSysGetAdapter 0000000180007098     asihpi64:ASIHPI64.dll
 0002:000000a0       __imp_HPI_AdapterOpen      00000001800070a0     asihpi64:ASIHPI64.dll
 0002:000000a8       __imp_HPI_MixerOpen        00000001800070a8     asihpi64:ASIHPI64.dll
 0002:000000b0       __imp_HPI_MixerClose       00000001800070b0     asihpi64:ASIHPI64.dll
 0002:000000b8       __imp_HPI_AdapterClose     00000001800070b8     asihpi64:ASIHPI64.dll
 0002:000000c0       __imp_HPI_SubSysCreate     00000001800070c0     asihpi64:ASIHPI64.dll
 0002:000000c8       __imp_HPI_SubSysGetNumAdapters 00000001800070c8     asihpi64:ASIHPI64.dll
 0002:000000d0       __imp_HPI_Object_ParameterHandle 00000001800070d0     asihpi64:ASIHPI64.dll
 0002:000000d8       __imp_HPI_SampleClock_GetLocalRate 00000001800070d8     asihpi64:ASIHPI64.dll
 0002:000000e0       __imp_HPI_MixerGetControl  00000001800070e0     asihpi64:ASIHPI64.dll
 0002:000000e8       __imp_HPI_SampleClock_SetLocalRate 00000001800070e8     asihpi64:ASIHPI64.dll
 0002:000000f0       \177ASIHPI64_NULL_THUNK_DATA 00000001800070f0     asihpi64:ASIHPI64.dll
 0002:000000f8       __imp_SetWindowSubclass    00000001800070f8     Comctl32:COMCTL32.dll
 0002:00000100       __imp_DefSubclassProc      0000000180007100     Comctl32:COMCTL32.dll
 0002:00000108       \177COMCTL32_NULL_THUNK_DATA 0000000180007108     Comctl32:COMCTL32.dll
 0002:00000110       __imp_CreateSolidBrush     0000000180007110     gdi32:GDI32.dll
 0002:00000118       __imp_BitBlt               0000000180007118     gdi32:GDI32.dll
 0002:00000120       __imp_GetTextMetricsW      0000000180007120     gdi32:GDI32.dll
 0002:00000128       __imp_GetTextFaceW         0000000180007128     gdi32:GDI32.dll
 0002:00000130       __imp_CreateFontIndirectW  0000000180007130     gdi32:GDI32.dll
 0002:00000138       __imp_SelectObject         0000000180007138     gdi32:GDI32.dll
 0002:00000140       \177GDI32_NULL_THUNK_DATA  0000000180007140     gdi32:GDI32.dll
 0002:00000148       __imp_GetLastError         0000000180007148     kernel32:KERNEL32.dll
 0002:00000150       __imp_EncodePointer        0000000180007150     kernel32:KERNEL32.dll
 0002:00000158       __imp_DecodePointer        0000000180007158     kernel32:KERNEL32.dll
 0002:00000160       __imp_IsDebuggerPresent    0000000180007160     kernel32:KERNEL32.dll
 0002:00000168       __imp_IsProcessorFeaturePresent 0000000180007168     kernel32:KERNEL32.dll
 0002:00000170       __imp_QueryPerformanceCounter 0000000180007170     kernel32:KERNEL32.dll
 0002:00000178       __imp_GetCurrentProcessId  0000000180007178     kernel32:KERNEL32.dll
 0002:00000180       __imp_GlobalFree           0000000180007180     kernel32:KERNEL32.dll
 0002:00000188       __imp_DisableThreadLibraryCalls 0000000180007188     kernel32:KERNEL32.dll
 0002:00000190       __imp_GetCurrentProcess    0000000180007190     kernel32:KERNEL32.dll
 0002:00000198       __imp_GetCurrentThreadId   0000000180007198     kernel32:KERNEL32.dll
 0002:000001a0       __imp_GlobalAlloc          00000001800071a0     kernel32:KERNEL32.dll
 0002:000001a8       __imp_GetSystemTimeAsFileTime 00000001800071a8     kernel32:KERNEL32.dll
 0002:000001b0       \177KERNEL32_NULL_THUNK_DATA 00000001800071b0     kernel32:KERNEL32.dll
 0002:000001b8       __imp__amsg_exit           00000001800071b8     MSVCRT:MSVCR120.dll
 0002:000001c0       __imp_free                 00000001800071c0     MSVCRT:MSVCR120.dll
 0002:000001c8       __imp_exit                 00000001800071c8     MSVCRT:MSVCR120.dll
 0002:000001d0       __imp__vswprintf_c_l       00000001800071d0     MSVCRT:MSVCR120.dll
 0002:000001d8       __imp_??2@YAPEAX_K@Z       00000001800071d8     MSVCRT:MSVCR120.dll
 0002:000001e0       __imp_??3@YAXPEAX@Z        00000001800071e0     MSVCRT:MSVCR120.dll
 0002:000001e8       __imp_memset               00000001800071e8     MSVCRT:MSVCR120.dll
 0002:000001f0       __imp__swprintf            00000001800071f0     MSVCRT:MSVCR120.dll
 0002:000001f8       __imp__wcsicmp             00000001800071f8     MSVCRT:MSVCR120.dll
 0002:00000200       __imp__malloc_crt          0000000180007200     MSVCRT:MSVCR120.dll
 0002:00000208       __imp__initterm            0000000180007208     MSVCRT:MSVCR120.dll
 0002:00000210       __imp__initterm_e          0000000180007210     MSVCRT:MSVCR120.dll
 0002:00000218       __imp___C_specific_handler 0000000180007218     MSVCRT:MSVCR120.dll
 0002:00000220       __imp___crt_debugger_hook  0000000180007220     MSVCRT:MSVCR120.dll
 0002:00000228       __imp___crtUnhandledException 0000000180007228     MSVCRT:MSVCR120.dll
 0002:00000230       __imp___crtTerminateProcess 0000000180007230     MSVCRT:MSVCR120.dll
 0002:00000238       __imp___crtCapturePreviousContext 0000000180007238     MSVCRT:MSVCR120.dll
 0002:00000240       __imp__lock                0000000180007240     MSVCRT:MSVCR120.dll
 0002:00000248       __imp__unlock              0000000180007248     MSVCRT:MSVCR120.dll
 0002:00000250       __imp__calloc_crt          0000000180007250     MSVCRT:MSVCR120.dll
 0002:00000258       __imp__onexit              0000000180007258     MSVCRT:MSVCR120.dll
 0002:00000260       __imp___clean_type_info_names_internal 0000000180007260     MSVCRT:MSVCR120.dll
 0002:00000268       __imp___CppXcptFilter      0000000180007268     MSVCRT:MSVCR120.dll
 0002:00000270       __imp___CxxFrameHandler3   0000000180007270     MSVCRT:MSVCR120.dll
 0002:00000278       __imp_memcpy               0000000180007278     MSVCRT:MSVCR120.dll
 0002:00000280       __imp___dllonexit          0000000180007280     MSVCRT:MSVCR120.dll
 0002:00000288       \177MSVCR120_NULL_THUNK_DATA 0000000180007288     MSVCRT:MSVCR120.dll
 0002:00000290       __imp_SetupDiGetClassDevsW 0000000180007290     Setupapi:SETUPAPI.dll
 0002:00000298       __imp_SetupDiOpenDevRegKey 0000000180007298     Setupapi:SETUPAPI.dll
 0002:000002a0       __imp_SetupDiDestroyDeviceInfoList 00000001800072a0     Setupapi:SETUPAPI.dll
 0002:000002a8       __imp_SetupDiEnumDeviceInfo 00000001800072a8     Setupapi:SETUPAPI.dll
 0002:000002b0       \177SETUPAPI_NULL_THUNK_DATA 00000001800072b0     Setupapi:SETUPAPI.dll
 0002:000002b8       __imp_SetWindowLongPtrW    00000001800072b8     user32:USER32.dll
 0002:000002c0       __imp_SetWindowPos         00000001800072c0     user32:USER32.dll
 0002:000002c8       __imp_GetWindowLongPtrW    00000001800072c8     user32:USER32.dll
 0002:000002d0       __imp_ScreenToClient       00000001800072d0     user32:USER32.dll
 0002:000002d8       __imp_SetDlgItemInt        00000001800072d8     user32:USER32.dll
 0002:000002e0       __imp_SetDlgItemTextW      00000001800072e0     user32:USER32.dll
 0002:000002e8       __imp_SetWindowTextW       00000001800072e8     user32:USER32.dll
 0002:000002f0       __imp_ShowWindow           00000001800072f0     user32:USER32.dll
 0002:000002f8       __imp_ScrollWindowEx       00000001800072f8     user32:USER32.dll
 0002:00000300       __imp_ClientToScreen       0000000180007300     user32:USER32.dll
 0002:00000308       __imp_SetScrollInfo        0000000180007308     user32:USER32.dll
 0002:00000310       __imp_EndDialog            0000000180007310     user32:USER32.dll
 0002:00000318       __imp_SendDlgItemMessageW  0000000180007318     user32:USER32.dll
 0002:00000320       __imp_EnableWindow         0000000180007320     user32:USER32.dll
 0002:00000328       __imp_CheckRadioButton     0000000180007328     user32:USER32.dll
 0002:00000330       __imp_DialogBoxParamW      0000000180007330     user32:USER32.dll
 0002:00000338       __imp_GetWindowRect        0000000180007338     user32:USER32.dll
 0002:00000340       __imp_GetDesktopWindow     0000000180007340     user32:USER32.dll
 0002:00000348       __imp_GetDlgItem           0000000180007348     user32:USER32.dll
 0002:00000350       __imp_IsWindowEnabled      0000000180007350     user32:USER32.dll
 0002:00000358       __imp_CallNextHookEx       0000000180007358     user32:USER32.dll
 0002:00000360       __imp_SendInput            0000000180007360     user32:USER32.dll
 0002:00000368       __imp_UnhookWindowsHookEx  0000000180007368     user32:USER32.dll
 0002:00000370       __imp_SetWindowsHookExW    0000000180007370     user32:USER32.dll
 0002:00000378       __imp_ReleaseDC            0000000180007378     user32:USER32.dll
 0002:00000380       __imp_GetDC                0000000180007380     user32:USER32.dll
 0002:00000388       __imp_SendMessageW         0000000180007388     user32:USER32.dll
 0002:00000390       __imp_MessageBoxW          0000000180007390     user32:USER32.dll
 0002:00000398       __imp_InvalidateRect       0000000180007398     user32:USER32.dll
 0002:000003a0       __imp_GetClientRect        00000001800073a0     user32:USER32.dll
 0002:000003a8       __imp_IsDlgButtonChecked   00000001800073a8     user32:USER32.dll
 0002:000003b0       __imp_LoadStringW          00000001800073b0     user32:USER32.dll
 0002:000003b8       __imp_DialogBoxIndirectParamW 00000001800073b8     user32:USER32.dll
 0002:000003c0       __imp_ExitWindowsEx        00000001800073c0     user32:USER32.dll
 0002:000003c8       __imp_GetDlgItemInt        00000001800073c8     user32:USER32.dll
 0002:000003d0       \177USER32_NULL_THUNK_DATA 00000001800073d0     user32:USER32.dll
 0002:000003d8       __xc_a                     00000001800073d8     MSVCRT:cinitexe.obj
 0002:000003e0       __xc_z                     00000001800073e0     MSVCRT:cinitexe.obj
 0002:000003e8       __xi_a                     00000001800073e8     MSVCRT:cinitexe.obj
 0002:00000400       __xi_z                     0000000180007400     MSVCRT:cinitexe.obj
 0002:00000410       GUID_DEVCLASS_MEDIA        0000000180007410     uuid:cguid_i.obj
 0002:00000420       _pRawDllMain               0000000180007420     MSVCRT:crtdll.obj
 0002:00000420       _pDefaultRawDllMain        0000000180007420     MSVCRT:crtdll.obj
 0002:00000438       ??_C@_1BI@IDMJHIIF@?$AAD?$AAe?$AAf?$AAa?$AAu?$AAl?$AAt?$AAI?$AAc?$AAo?$AAn?$AA?$AA@ 0000000180007438     CtrlPnlReg.obj
 0002:00000450       ??_C@_1M@JLDCNMKN@?$AAS?$AAh?$AAe?$AAl?$AAl?$AA?$AA@ 0000000180007450     CtrlPnlReg.obj
 0002:00000460       ??_C@_1BA@MGKEIBAA@?$AAC?$AAo?$AAm?$AAm?$AAa?$AAn?$AAd?$AA?$AA@ 0000000180007460     CtrlPnlReg.obj
 0002:00000470       ??_C@_1CA@KMFDEJAN@?$AAL?$AAo?$AAc?$AAa?$AAl?$AAi?$AAz?$AAe?$AAd?$AAS?$AAt?$AAr?$AAi?$AAn?$AAg?$AA?$AA@ 0000000180007470     CtrlPnlReg.obj
 0002:00000490       ??_C@_1BA@NFCMADAA@?$AAI?$AAn?$AAf?$AAo?$AAT?$AAi?$AAp?$AA?$AA@ 0000000180007490     CtrlPnlReg.obj
 0002:000004a0       ??_C@_1CO@MIJIOHLE@?$AAS?$AAy?$AAs?$AAt?$AAe?$AAm?$AA?4?$AAA?$AAp?$AAp?$AAl?$AAi?$AAc?$AAa?$AAt?$AAi?$AAo?$AAn?$AAN?$AAa?$AAm?$AAe?$AA?$AA@ 00000001800074a0     CtrlPnlReg.obj
 0002:000004d0       ??_C@_1DK@DDDACLHP@?$AAS?$AAy?$AAs?$AAt?$AAe?$AAm?$AA?4?$AAC?$AAo?$AAn?$AAt?$AAr?$AAo?$AAl?$AAP?$AAa?$AAn?$AAe?$AAl?$AA?4?$AAC?$AAa?$AAt?$AAe?$AAg?$AAo?$AAr?$AAy?$AA?$AA@ 00000001800074d0     CtrlPnlReg.obj
 0002:00000510       ??_C@_1M@KANJNLFF@?$AAC?$AAL?$AAS?$AAI?$AAD?$AA?$AA@ 0000000180007510     CtrlPnlReg.obj
 0002:00000520       ??_C@_1JE@KFOKPFDN@?$AAS?$AAO?$AAF?$AAT?$AAW?$AAA?$AAR?$AAE?$AA?2?$AAM?$AAi?$AAc?$AAr?$AAo?$AAs?$AAo?$AAf?$AAt?$AA?2?$AAW?$AAi?$AAn?$AAd?$AAo?$AAw?$AAs?$AA?2?$AAC?$AAu?$AAr?$AAr?$AAe@ 0000000180007520     CtrlPnlReg.obj
 0002:000005b8       ??_C@_1BC@PKEHKAEB@?$AAE?$AAx?$AAp?$AAl?$AAo?$AAr?$AAe?$AAr?$AA?$AA@ 00000001800075b8     CtrlPnlReg.obj
 0002:000005d0       ??_C@_1BI@DMHEGHBF@?$AAD?$AAi?$AAs?$AAa?$AAl?$AAl?$AAo?$AAw?$AAC?$AAp?$AAl?$AA?$AA@ 00000001800075d0     CtrlPnlReg.obj
 0002:000005f0       ??_C@_1GG@IPMCGENI@?$AAS?$AAO?$AAF?$AAT?$AAW?$AAA?$AAR?$AAE?$AA?2?$AAM?$AAi?$AAc?$AAr?$AAo?$AAs?$AAo?$AAf?$AAt?$AA?2?$AAW?$AAi?$AAn?$AAd?$AAo?$AAw?$AAs?$AA?2?$AAC?$AAu?$AAr?$AAr?$AAe@ 00000001800075f0     CtrlPnlReg.obj
 0002:00000658       ??_C@_15KNBIKKIN@?$AA?$CF?$AAd?$AA?$AA@ 0000000180007658     CtrlPnlReg.obj
 0002:00000660       ??_C@_1M@DMOFNHON@?$AAR?$AAu?$AAn?$AAA?$AAs?$AA?$AA@ 0000000180007660     CtrlPnlReg.obj
 0002:00000670       ??_C@_1JA@EMBPJHGA@?$AAS?$AAO?$AAF?$AAT?$AAW?$AAA?$AAR?$AAE?$AA?2?$AAM?$AAi?$AAc?$AAr?$AAo?$AAs?$AAo?$AAf?$AAt?$AA?2?$AAW?$AAi?$AAn?$AAd?$AAo?$AAw?$AAs?$AA?2?$AAC?$AAu?$AAr?$AAr?$AAe@ 0000000180007670     CtrlPnlReg.obj
 0002:00000704       ?m_initial_count@quick_conflict_detector@@0HB 0000000180007704     AdapterInfo.obj
 0002:00000708       ?m_bits_per_entry@quick_conflict_detector@@0HB 0000000180007708     AdapterInfo.obj
 0002:00000710       ??_C@_1CK@PCFIAPBJ@?$AAC?$AAh?$AAa?$AAn?$AAn?$AAe?$AAl?$AAs?$AAP?$AAe?$AAr?$AAS?$AAu?$AAb?$AAd?$AAe?$AAv?$AAi?$AAc?$AAe?$AA?$AA@ 0000000180007710     AdapterInfo.obj
 0002:00000740       ??_C@_07DMJBFPJJ@Channel?$AA@ 0000000180007740     AdapterInfo.obj
 0002:00000748       ??_C@_1DG@LNIOOGGI@?$AAH?$AAP?$AAI?$AA_?$AAO?$AAb?$AAj?$AAe?$AAc?$AAt?$AA_?$AAP?$AAa?$AAr?$AAa?$AAm?$AAe?$AAt?$AAe?$AAr?$AAH?$AAa?$AAn?$AAd?$AAl?$AAe?$AA?$AA@ 0000000180007748     AdapterInfo.obj
 0002:00000780       ??_C@_1EE@PDNLGPFH@?$AAF?$AAu?$AAn?$AAc?$AAt?$AAi?$AAo?$AAn?$AA?3?$AA?5?$AA?$CC?$AA?$CF?$AAs?$AA?$CC?$AA?5?$AAr?$AAe?$AAt?$AAu?$AAr?$AAn?$AAe?$AAd?$AA?5?$AAe?$AAr?$AAr?$AAo?$AAr?$AA?3?$AA?5?$AA?$CF@ 0000000180007780     AdapterInfo.obj
 0002:000007c8       ??_C@_1CG@EPCCAABM@?$AAH?$AAP?$AAI?$AA_?$AAO?$AAb?$AAj?$AAe?$AAc?$AAt?$AA_?$AAG?$AAe?$AAt?$AAI?$AAn?$AAf?$AAo?$AA?$AA@ 00000001800077c8     AdapterInfo.obj
 0002:000007f0       ??_C@_1CK@OJGCMPLE@?$AAe?$AAn?$AAt?$AAi?$AAt?$AAy?$AA?5?$AAn?$AAo?$AAt?$AA?5?$AAw?$AAr?$AAi?$AAt?$AAe?$AAa?$AAb?$AAl?$AAe?$AA?$AA@ 00000001800077f0     AdapterInfo.obj
 0002:00000820       ??_C@_1DE@CHMJBILK@?$AAH?$AAP?$AAI?$AA_?$AAO?$AAb?$AAj?$AAe?$AAc?$AAt?$AA_?$AAG?$AAe?$AAt?$AAV?$AAa?$AAl?$AAu?$AAe?$AAE?$AAn?$AAt?$AAi?$AAt?$AAy?$AA?$AA@ 0000000180007820     AdapterInfo.obj
 0002:00000858       ??_C@_1CE@IIDJKCDC@?$AAH?$AAP?$AAI?$AA_?$AAU?$AAn?$AAi?$AAv?$AAe?$AAr?$AAs?$AAa?$AAl?$AA_?$AAS?$AAe?$AAt?$AA?$AA@ 0000000180007858     AdapterInfo.obj
 0002:00000880       ??_C@_1DA@MIHDLDAM@?$AAH?$AAP?$AAI?$AA_?$AAE?$AAn?$AAt?$AAi?$AAt?$AAy?$AA_?$AAA?$AAl?$AAl?$AAo?$AAc?$AAA?$AAn?$AAd?$AAP?$AAa?$AAc?$AAk?$AA?$AA@ 0000000180007880     AdapterInfo.obj
 0002:000008b0       ??_C@_1CA@BDNGJNOP@?$AAt?$AAy?$AAp?$AAe?$AA?5?$AAi?$AAs?$AA?5?$AAn?$AAo?$AAt?$AA?5?$AAi?$AAn?$AAt?$AA?$AA@ 00000001800078b0     AdapterInfo.obj
 0002:000008d0       ??_C@_1CA@DLBCANMK@?$AAH?$AAP?$AAI?$AAA?$AAd?$AAa?$AAp?$AAt?$AAe?$AAr?$AAI?$AAn?$AAd?$AAe?$AAx?$AA?$AA@ 00000001800078d0     AdapterInfo.obj
 0002:000008f0       ??_C@_1O@GAOCKAOK@?$AAD?$AAr?$AAi?$AAv?$AAe?$AAr?$AA?$AA@ 00000001800078f0     AdapterInfo.obj
 0002:00000900       ??_C@_1BK@CJIHEDPJ@?$AAa?$AAs?$AAi?$AAw?$AAd?$AAm?$AAx?$AAv?$AA?4?$AAs?$AAy?$AAs?$AA?$AA@ 0000000180007900     AdapterInfo.obj
 0002:00000920       ??_C@_1BK@HPPNMIOH@?$AAa?$AAs?$AAi?$AAw?$AAd?$AAm?$AA6?$AA4?$AA?4?$AAs?$AAy?$AAs?$AA?$AA@ 0000000180007920     AdapterInfo.obj
 0002:00000940       ??_C@_1IM@DLGGPNPG@?$AAr?$AAu?$AAn?$AAd?$AAl?$AAl?$AA3?$AA2?$AA?5?$AA?$CF?$AAS?$AAy?$AAs?$AAt?$AAe?$AAm?$AAR?$AAo?$AAo?$AAt?$AA?$CF?$AA?2?$AAs?$AAy?$AAs?$AAt?$AAe?$AAm?$AA3?$AA2?$AA?2?$AAA@ 0000000180007940     BluLinkCfg.obj
 0002:000009d0       ??_C@_1FE@EPNOENEO@?$AA?$CF?$AAS?$AAy?$AAs?$AAt?$AAe?$AAm?$AAR?$AAo?$AAo?$AAt?$AA?$CF?$AA?2?$AAs?$AAy?$AAs?$AAt?$AAe?$AAm?$AA3?$AA2?$AA?2?$AAA?$AAs?$AAi?$AAB?$AAl?$AAC?$AAf?$AAg?$AA6?$AA4@ 00000001800079d0     BluLinkCfg.obj
 0002:00000a28       ??_C@_17BIMEGBJF@?$AA2?$AA?0?$AA8?$AA?$AA@ 0000000180007a28     BluLinkCfg.obj
 0002:00000a30       ??_C@_1CM@EGHHJIBM@?$AAA?$AAu?$AAd?$AAi?$AAo?$AAS?$AAc?$AAi?$AAe?$AAn?$AAc?$AAe?$AA?4?$AAA?$AAs?$AAi?$AAB?$AAl?$AAC?$AAf?$AAg?$AA?$AA@ 0000000180007a30     BluLinkCfg.obj
 0002:00000a60       ??_C@_1HC@EGCIGHEM@?$AAC?$AAo?$AAn?$AAf?$AAi?$AAg?$AAu?$AAr?$AAe?$AA?5?$AAB?$AAL?$AAU?$AA?5?$AAl?$AAi?$AAn?$AAk?$AA?5?$AAi?$AAn?$AAp?$AAu?$AAt?$AA?5?$AAa?$AAn?$AAd?$AA?5?$AAo?$AAu?$AAt@ 0000000180007a60     BluLinkCfg.obj
 0002:00000ad8       ??_C@_1CO@OMKBIMF@?$AAB?$AAL?$AAU?$AA?5?$AAl?$AAi?$AAn?$AAk?$AA?5?$AAC?$AAo?$AAn?$AAf?$AAi?$AAg?$AAu?$AAr?$AAa?$AAt?$AAi?$AAo?$AAn?$AA?$AA@ 0000000180007ad8     BluLinkCfg.obj
 0002:00000b10       ??_C@_1EI@IPMPPGE@?$AAA?$AAu?$AAd?$AAi?$AAo?$AAS?$AAc?$AAi?$AAe?$AAn?$AAc?$AAe?$AA?5?$AAB?$AAL?$AAU?$AA?5?$AAl?$AAi?$AAn?$AAk?$AA?5?$AAC?$AAo?$AAn?$AAt?$AAr?$AAo?$AAl?$AA?5?$AAP?$AAa@ 0000000180007b10     BluLinkCfg.obj
 0002:00000b60       ??_C@_1EO@GGPFOMEM@?$AA?$HL?$AA7?$AAC?$AAC?$AAC?$AAF?$AA9?$AA7?$AA3?$AA?9?$AA9?$AA5?$AAF?$AA2?$AA?9?$AA4?$AAf?$AA5?$AAe?$AA?9?$AA8?$AA5?$AA7?$AA3?$AA?9?$AA9?$AA5?$AA3?$AA9?$AA3?$AAB?$AAD@ 0000000180007b60     BluLinkCfg.obj
 0002:00000bb0       ??_C@_1BO@MAGCHMCB@?$AAA?$AAs?$AAi?$AAB?$AAl?$AAC?$AAf?$AAg?$AA6?$AA4?$AA?4?$AAd?$AAl?$AAl?$AA?$AA@ 0000000180007bb0     BluLinkCfg.obj
 0002:00000bd0       ??_C@_1EA@LCPOBPC@?$AAN?$AAo?$AA?5?$AAB?$AAL?$AAU?$AA?5?$AAl?$AAi?$AAn?$AAk?$AA?5?$AAa?$AAd?$AAa?$AAp?$AAt?$AAe?$AAr?$AAs?$AA?5?$AAw?$AAe?$AAr?$AAe?$AA?5?$AAf?$AAo?$AAu?$AAn?$AAd?$AA?$AA@ 0000000180007bd0     BluLinkCfg.obj
 0002:00000c10       ??_C@_1BK@EAIFNPAP@?$AAA?$AAs?$AAi?$AAB?$AAl?$AAC?$AAf?$AAg?$AA?4?$AAd?$AAl?$AAl?$AA?$AA@ 0000000180007c10     ConfigDialog.obj
 0002:00000c30       ??_C@_1EK@CCCKMOMP@?$AAE?$AAr?$AAr?$AA?5?$AA?9?$AA?5?$AAm?$AAu?$AAl?$AAt?$AAi?$AAp?$AAl?$AAe?$AA?5?$AAK?$AAe?$AAy?$AAb?$AAo?$AAa?$AAr?$AAd?$AAH?$AAo?$AAo?$AAk?$AA?5?$AAo?$AAb?$AAj?$AAe@ 0000000180007c30     ConfigDialog.obj
 0002:00000c80       ??_C@_1HM@MOHNHKHM@?$AAY?$AAo?$AAu?$AA?5?$AAm?$AAu?$AAs?$AAt?$AA?5?$AAr?$AAe?$AAb?$AAo?$AAo?$AAt?$AA?5?$AAy?$AAo?$AAu?$AAr?$AA?5?$AAc?$AAo?$AAm?$AAp?$AAu?$AAt?$AAe?$AAr?$AA?5?$AAf?$AAo@ 0000000180007c80     ConfigDialog.obj
 0002:00000d00       ??_C@_1MK@ILLPMKJC@?$AAY?$AAo?$AAu?$AA?5?$AAm?$AAu?$AAs?$AAt?$AA?5?$AAr?$AAe?$AAb?$AAo?$AAo?$AAt?$AA?5?$AAy?$AAo?$AAu?$AAr?$AA?5?$AAc?$AAo?$AAm?$AAp?$AAu?$AAt?$AAe?$AAr?$AA?5?$AAt?$AAo@ 0000000180007d00     ConfigDialog.obj
 0002:00000dd0       ??_C@_1IK@MCLDGMBA@?$AAA?$AAd?$AAa?$AAp?$AAt?$AAe?$AAr?$AAs?$AA?5?$AAh?$AAa?$AAv?$AAe?$AA?5?$AAd?$AAi?$AAf?$AAf?$AAe?$AAr?$AAe?$AAn?$AAt?$AA?5?$AAs?$AAa?$AAm?$AAp?$AAl?$AAe?$AAr?$AAa@ 0000000180007dd0     ConfigDialog.obj
 0002:00000e60       ??_C@_1LI@EINHHKMF@?$AAA?$AAd?$AAa?$AAp?$AAt?$AAe?$AAr?$AAs?$AA?5?$AAh?$AAa?$AAv?$AAe?$AA?5?$AAd?$AAi?$AAf?$AAf?$AAe?$AAr?$AAe?$AAn?$AAt?$AA?5?$AAW?$AAD?$AAM?$AA?5?$AAd?$AAe?$AAv?$AAi@ 0000000180007e60     ConfigDialog.obj
 0002:00000f20       ??_C@_1GI@JONNNMHI@?$AAS?$AAo?$AAm?$AAe?$AA?5?$AAc?$AAh?$AAa?$AAn?$AAn?$AAe?$AAl?$AA?5?$AAs?$AAe?$AAt?$AAt?$AAi?$AAn?$AAg?$AAs?$AA?5?$AAn?$AAo?$AAt?$AA?5?$AAa?$AAp?$AAp?$AAl?$AAi?$AAe@ 0000000180007f20     ConfigDialog.obj
 0002:00000f88       ??_C@_15LNJDIFMI@?$AAI?$AAn?$AA?$AA@ 0000000180007f88     ConfigDialog.obj
 0002:00000f90       ??_C@_17NFNCFLGO@?$AAO?$AAu?$AAt?$AA?$AA@ 0000000180007f90     ConfigDialog.obj
 0002:00000f98       ??_C@_1DO@CFJJBDGO@?$AA?$CF?$AAd?$AA?5?$AA?9?$AA?5?$AAB?$AAL?$AAU?$AA?9?$AAP?$AAC?$AAI?$AA?5?$AAA?$AAS?$AAI?$AAO?$AA?5?$AA?$CF?$AAs?$AA?5?$AA?$CI?$AA?$CF?$AAd?$AA?5?$AA?9?$AA?5?$AA?$CF?$AAd?$AA?$CJ?$AA?$AA@ 0000000180007f98     ConfigDialog.obj
 0002:00000fe0       ??_C@_1EA@DMFCDEDA@?$AA?$CF?$AAd?$AA?5?$AA?9?$AA?5?$AAB?$AAL?$AAU?$AA?9?$AAP?$AAC?$AAI?$AA?1?$AA?$CF?$AAd?$AA?5?$AAW?$AAD?$AAM?$AA?5?$AA?$CF?$AAs?$AA?5?$AA?$CI?$AAd?$AAi?$AAr?$AAe?$AAc?$AAt?$AA?$CJ?$AA?$AA@ 0000000180007fe0     ConfigDialog.obj
 0002:00001020       ??_C@_1CA@LANDJAEG@?$AAC?$AAh?$AAa?$AAn?$AAn?$AAe?$AAl?$AA?5?$AAN?$AAu?$AAm?$AAb?$AAe?$AAr?$AA?3?$AA?$AA@ 0000000180008020     ConfigDialog.obj
 0002:00001040       ??_C@_15OEEJMLKJ@?$AA4?$AA8?$AA?$AA@ 0000000180008040     ConfigDialog.obj
 0002:00001048       ??_C@_15LIAIKPEE@?$AA9?$AA6?$AA?$AA@ 0000000180008048     ConfigDialog.obj
 0002:00001050       ??_C@_13JGCMLPCH@?$AA1?$AA?$AA@ 0000000180008050     ConfigDialog.obj
 0002:00001054       ??_C@_13IEJJBAMJ@?$AA2?$AA?$AA@ 0000000180008054     ConfigDialog.obj
 0002:00001058       ??_C@_13KBPCEPBF@?$AA4?$AA?$AA@ 0000000180008058     ConfigDialog.obj
 0002:0000105c       ??_C@_13OLCEPAKN@?$AA8?$AA?$AA@ 000000018000805c     ConfigDialog.obj
 0002:00001060       ??_C@_1LA@FFMJMMLD@?$AAC?$AAh?$AAa?$AAn?$AAg?$AAe?$AAs?$AA?5?$AAc?$AAa?$AAn?$AAn?$AAo?$AAt?$AA?5?$AAb?$AAe?$AA?5?$AAa?$AAp?$AAp?$AAl?$AAi?$AAe?$AAd?$AA?5?$AAb?$AAe?$AAc?$AAa?$AAu?$AAs@ 0000000180008060     ConfigDialog.obj
 0002:00001110       ??_C@_1CI@NKKEIBLI@?$AAS?$AAe?$AAS?$AAh?$AAu?$AAt?$AAd?$AAo?$AAw?$AAn?$AAP?$AAr?$AAi?$AAv?$AAi?$AAl?$AAe?$AAg?$AAe?$AA?$AA@ 0000000180008110     ConfigDialog.obj
 0002:00001138       ??_C@_17OMFOJHEJ@?$AAW?$AAT?$AAF?$AA?$AA@ 0000000180008138     ConfigDialog.obj
 0002:00001170       _load_config_used          0000000180008170     MSVCRT:loadcfg.obj
 0002:000011e0       __rtc_iaa                  00000001800081e0     MSVCRT:initsect.obj
 0002:000011e8       __rtc_izz                  00000001800081e8     MSVCRT:initsect.obj
 0002:000011f0       __rtc_taa                  00000001800081f0     MSVCRT:initsect.obj
 0002:000011f8       __rtc_tzz                  00000001800081f8     MSVCRT:initsect.obj
 0002:00001b80       __IMPORT_DESCRIPTOR_COMCTL32 0000000180008b80     Comctl32:COMCTL32.dll
 0002:00001b94       __IMPORT_DESCRIPTOR_SETUPAPI 0000000180008b94     Setupapi:SETUPAPI.dll
 0002:00001ba8       __IMPORT_DESCRIPTOR_ASIHPI64 0000000180008ba8     asihpi64:ASIHPI64.dll
 0002:00001bbc       __IMPORT_DESCRIPTOR_KERNEL32 0000000180008bbc     kernel32:KERNEL32.dll
 0002:00001bd0       __IMPORT_DESCRIPTOR_USER32 0000000180008bd0     user32:USER32.dll
 0002:00001be4       __IMPORT_DESCRIPTOR_GDI32  0000000180008be4     gdi32:GDI32.dll
 0002:00001bf8       __IMPORT_DESCRIPTOR_ADVAPI32 0000000180008bf8     advapi32:ADVAPI32.dll
 0002:00001c0c       __IMPORT_DESCRIPTOR_MSVCR120 0000000180008c0c     MSVCRT:MSVCR120.dll
 0002:00001c20       __NULL_IMPORT_DESCRIPTOR   0000000180008c20     Comctl32:COMCTL32.dll
 0003:00000000       __security_cookie          000000018000a000     MSVCRT:gs_cookie.obj
 0003:00000008       __security_cookie_complement 000000018000a008     MSVCRT:gs_cookie.obj
 0003:00000010       __native_dllmain_reason    000000018000a010     MSVCRT:natstart.obj
 0003:00000ca8       ?__type_info_root_node@@3U__type_info_node@@A 000000018000aca8     MSVCRT:tncleanup.obj
 0003:00000cc0       ?g_phSubSys@@3PEAUhpi_hsubsys@@EA 000000018000acc0     AdapterInfo.obj
 0003:00000cc8       ?hinstance@@3PEAUHINSTANCE__@@EA 000000018000acc8     BluLinkCfg.obj
 0003:00000cd0       ?hYellowBrush@@3PEAUHBRUSH__@@EA 000000018000acd0     ChanControl.obj
 0003:00000cd8       ?hGreenBrush@@3PEAUHBRUSH__@@EA 000000018000acd8     ChanControl.obj
 0003:00000ce0       ?hRedBrush@@3PEAUHBRUSH__@@EA 000000018000ace0     ChanControl.obj
 0003:00000ce8       ?m_focus@KeyboardHook@@0_NA 000000018000ace8     ConfigDialog.obj
 0003:00000cf0       ?szTitle@@3PA_WA           000000018000acf0     ConfigDialog.obj
 0003:00000db8       ?m_hkbhook@KeyboardHook@@0PEAUHHOOK__@@EA 000000018000adb8     ConfigDialog.obj
 0003:00000dc8       __@@_PchSym_@00@UzhrUhdUzkkhUyoformpxutUcGEUivovzhvUhgwzucOlyq@CF90FC38A5F78E7C 000000018000adc8     stdafx.obj
 0003:00000dd0       __native_startup_lock      000000018000add0     <common>
 0003:00000dd8       __native_startup_state     000000018000add8     <common>
 0003:00000de0       __onexitend                000000018000ade0     <common>
 0003:00000de8       __onexitbegin              000000018000ade8     <common>
 0003:00000df0       __dyn_tls_init_callback    000000018000adf0     <common>

 entry point at        0001:00004aec

 Static symbols

 0001:000027e0       swprintf                   00000001800037e0 f   * CIL library *:* CIL module *
 0001:000027e0       swprintf                   00000001800037e0 f   * CIL library *:* CIL module *
 0001:000037c0       $LN26                      00000001800047c0     * CIL library *:* CIL module *
 0001:00004810       $$000000                   0000000180005810     MSVCRT:amdsecgs.obj
 0001:00004840       pre_c_init                 0000000180005840 f   MSVCRT:crtdll.obj
 0001:00004b2c       __DllMainCRTStartup        0000000180005b2c f   MSVCRT:crtdll.obj
 0001:00005180       ?dtor$0@?0??RunDialog@@YAXPEAUHWND__@@_N@Z@4HA 0000000180006180 f   * CIL library *:* CIL module *
 0001:0000518c       ?dtor$1@?0??RunDialog@@YAXPEAUHWND__@@_N@Z@4HA 000000018000618c f   * CIL library *:* CIL module *
 0001:00005198       __DllMainCRTStartup$filt$0 0000000180006198 f   MSVCRT:crtdll.obj
 0001:000051bd       __DllMainCRTStartup$fin$1  00000001800061bd f   MSVCRT:crtdll.obj
 0001:000051e0       _IsNonwritableInCurrentImage$filt$0 00000001800061e0 f   MSVCRT:pesect.obj
 0001:00005200       _onexit$fin$0              0000000180006200 f   MSVCRT:atonexit.obj
 0002:000003f0       pcinit                     00000001800073f0     MSVCRT:crtdll.obj
 0002:000003f8       pinit                      00000001800073f8     MSVCRT:atonexit.obj
 0002:00000428       GS_ExceptionPointers       0000000180007428     MSVCRT:gs_report.obj
 0002:00000700       dwOne                      0000000180007700     * CIL library *:* CIL module *
 0002:00001140       $cppxdata$?RunDialog@@YAXPEAUHWND__@@_N@Z 0000000180008140     * CIL library *:* CIL module *
 0002:00001200       $unwind$?AddList@ControlPanelRegistration@@AEAA_NPEAUkey_path_entry@@PEAUreg_list_entry@@@Z 0000000180008200     * CIL library *:* CIL module *
 0002:0000120c       $chain$0$?AddList@ControlPanelRegistration@@AEAA_NPEAUkey_path_entry@@PEAUreg_list_entry@@@Z 000000018000820c     * CIL library *:* CIL module *
 0002:00001220       $chain$1$?AddList@ControlPanelRegistration@@AEAA_NPEAUkey_path_entry@@PEAUreg_list_entry@@@Z 0000000180008220     * CIL library *:* CIL module *
 0002:00001230       $chain$2$?AddList@ControlPanelRegistration@@AEAA_NPEAUkey_path_entry@@PEAUreg_list_entry@@@Z 0000000180008230     * CIL library *:* CIL module *
 0002:00001244       $unwind$?RemoveList@ControlPanelRegistration@@AEAA_NPEAUkey_path_entry@@PEAUreg_list_entry@@@Z 0000000180008244     * CIL library *:* CIL module *
 0002:00001250       $chain$0$?RemoveList@ControlPanelRegistration@@AEAA_NPEAUkey_path_entry@@PEAUreg_list_entry@@@Z 0000000180008250     * CIL library *:* CIL module *
 0002:00001264       $chain$1$?RemoveList@ControlPanelRegistration@@AEAA_NPEAUkey_path_entry@@PEAUreg_list_entry@@@Z 0000000180008264     * CIL library *:* CIL module *
 0002:00001274       $unwind$?FindValueName@ControlPanelRegistration@@AEAA_NPEAUHKEY__@@PEB_WPEA_WH@Z 0000000180008274     * CIL library *:* CIL module *
 0002:00001294       $unwind$?IsRegistered@ControlPanelRegistration@@QEAA?AW4CPRegState@@XZ 0000000180008294     * CIL library *:* CIL module *
 0002:000012a4       $unwind$?Register@ControlPanelRegistration@@QEAA_NXZ 00000001800082a4     * CIL library *:* CIL module *
 0002:000012a4       $unwind$?UnRegister@ControlPanelRegistration@@QEAA_NXZ 00000001800082a4     * CIL library *:* CIL module *
 0002:000012b0       $chain$2$?Register@ControlPanelRegistration@@QEAA_NXZ 00000001800082b0     * CIL library *:* CIL module *
 0002:000012cc       $chain$3$?Register@ControlPanelRegistration@@QEAA_NXZ 00000001800082cc     * CIL library *:* CIL module *
 0002:000012dc       $chain$2$?UnRegister@ControlPanelRegistration@@QEAA_NXZ 00000001800082dc     * CIL library *:* CIL module *
 0002:000012f8       $chain$3$?UnRegister@ControlPanelRegistration@@QEAA_NXZ 00000001800082f8     * CIL library *:* CIL module *
 0002:00001308       $unwind$?Show@ControlPanelRegistration@@QEAA_N_N@Z 0000000180008308     * CIL library *:* CIL module *
 0002:00001320       $chain$0$?Show@ControlPanelRegistration@@QEAA_N_N@Z 0000000180008320     * CIL library *:* CIL module *
 0002:00001334       $chain$1$?Show@ControlPanelRegistration@@QEAA_N_N@Z 0000000180008334     * CIL library *:* CIL module *
 0002:00001344       $unwind$?SetChannel@BluLinkChannelControl@@QEAAXH@Z 0000000180008344     * CIL library *:* CIL module *
 0002:00001344       $unwind$?SetConflict@BluLinkChannelControl@@QEAAXPEAV1@@Z 0000000180008344     * CIL library *:* CIL module *
 0002:00001354       $unwind$?SetChannelsPerDevice@DialogParameters@@QEAAXH@Z 0000000180008354     * CIL library *:* CIL module *
 0002:0000135c       $chain$0$?SetChannelsPerDevice@DialogParameters@@QEAAXH@Z 000000018000835c     * CIL library *:* CIL module *
 0002:00001370       $chain$1$?SetChannelsPerDevice@DialogParameters@@QEAAXH@Z 0000000180008370     * CIL library *:* CIL module *
 0002:00001380       $unwind$?AllocateBlulinkControls@DialogParameters@@QEAAXXZ 0000000180008380     * CIL library *:* CIL module *
 0002:00001388       $chain$0$?AllocateBlulinkControls@DialogParameters@@QEAAXXZ 0000000180008388     * CIL library *:* CIL module *
 0002:0000139c       $chain$2$?AllocateBlulinkControls@DialogParameters@@QEAAXXZ 000000018000839c     * CIL library *:* CIL module *
 0002:000013b4       $chain$3$?AllocateBlulinkControls@DialogParameters@@QEAAXXZ 00000001800083b4     * CIL library *:* CIL module *
 0002:000013c8       $chain$4$?AllocateBlulinkControls@DialogParameters@@QEAAXXZ 00000001800083c8     * CIL library *:* CIL module *
 0002:000013d8       $chain$5$?AllocateBlulinkControls@DialogParameters@@QEAAXXZ 00000001800083d8     * CIL library *:* CIL module *
 0002:000013e8       $unwind$?FoundAsiRegistryKey@AsiBluLinkConfigPerAdapterInfo@@QEAAHPEAVDialogParameters@@PEAUHKEY__@@@Z 00000001800083e8     * CIL library *:* CIL module *
 0002:000013f4       $unwind$?GetChannelFromHpiControl@@YAHII@Z 00000001800083f4     * CIL library *:* CIL module *
 0002:00001408       $unwind$?InitChannels@AsiBluLinkConfigPerAdapterInfo@@QEAAXPEAVDialogParameters@@PEAX@Z 0000000180008408     * CIL library *:* CIL module *
 0002:00001418       $chain$2$?InitChannels@AsiBluLinkConfigPerAdapterInfo@@QEAAXPEAVDialogParameters@@PEAX@Z 0000000180008418     * CIL library *:* CIL module *
 0002:00001434       $chain$3$?InitChannels@AsiBluLinkConfigPerAdapterInfo@@QEAAXPEAVDialogParameters@@PEAX@Z 0000000180008434     * CIL library *:* CIL module *
 0002:00001444       $unwind$?SaveChannelToHpiControl@@YAXIIH@Z 0000000180008444     * CIL library *:* CIL module *
 0002:00001458       $unwind$?SaveChannels@AsiBluLinkConfigPerAdapterInfo@@QEAAXPEAVDialogParameters@@PEAX@Z 0000000180008458     * CIL library *:* CIL module *
 0002:00001460       $chain$0$?SaveChannels@AsiBluLinkConfigPerAdapterInfo@@QEAAXPEAVDialogParameters@@PEAX@Z 0000000180008460     * CIL library *:* CIL module *
 0002:00001474       $chain$6$?SaveChannels@AsiBluLinkConfigPerAdapterInfo@@QEAAXPEAVDialogParameters@@PEAX@Z 0000000180008474     * CIL library *:* CIL module *
 0002:0000149c       $chain$7$?SaveChannels@AsiBluLinkConfigPerAdapterInfo@@QEAAXPEAVDialogParameters@@PEAX@Z 000000018000849c     * CIL library *:* CIL module *
 0002:000014bc       $chain$8$?SaveChannels@AsiBluLinkConfigPerAdapterInfo@@QEAAXPEAVDialogParameters@@PEAX@Z 00000001800084bc     * CIL library *:* CIL module *
 0002:000014cc       $unwind$?FoundAsiRegistryKey@AsiBluLinkConfigAdapterInfo@@AEAAHPEAVDialogParameters@@PEAUHKEY__@@@Z 00000001800084cc     * CIL library *:* CIL module *
 0002:000014e0       $unwind$?InitChannelsPerDevice@AsiBluLinkConfigAdapterInfo@@AEAAXPEAVDialogParameters@@PEAUHWND__@@@Z 00000001800084e0     * CIL library *:* CIL module *
 0002:000014f8       $chain$2$?InitChannelsPerDevice@AsiBluLinkConfigAdapterInfo@@AEAAXPEAVDialogParameters@@PEAUHWND__@@@Z 00000001800084f8     * CIL library *:* CIL module *
 0002:00001514       $chain$3$?InitChannelsPerDevice@AsiBluLinkConfigAdapterInfo@@AEAAXPEAVDialogParameters@@PEAUHWND__@@@Z 0000000180008514     * CIL library *:* CIL module *
 0002:00001528       $chain$4$?InitChannelsPerDevice@AsiBluLinkConfigAdapterInfo@@AEAAXPEAVDialogParameters@@PEAUHWND__@@@Z 0000000180008528     * CIL library *:* CIL module *
 0002:00001538       $chain$5$?InitChannelsPerDevice@AsiBluLinkConfigAdapterInfo@@AEAAXPEAVDialogParameters@@PEAUHWND__@@@Z 0000000180008538     * CIL library *:* CIL module *
 0002:00001548       $chain$6$?InitChannelsPerDevice@AsiBluLinkConfigAdapterInfo@@AEAAXPEAVDialogParameters@@PEAUHWND__@@@Z 0000000180008548     * CIL library *:* CIL module *
 0002:00001568       $unwind$?InitAdapterInfo@AsiBluLinkConfigAdapterInfo@@QEAAHPEAVDialogParameters@@PEAUHWND__@@_N@Z 0000000180008568     * CIL library *:* CIL module *
 0002:0000158c       $unwind$?SaveAdapterInfo@AsiBluLinkConfigAdapterInfo@@QEAAXPEAVDialogParameters@@_N@Z 000000018000858c     * CIL library *:* CIL module *
 0002:000015a0       $chain$1$?SaveAdapterInfo@AsiBluLinkConfigAdapterInfo@@QEAAXPEAVDialogParameters@@_N@Z 00000001800085a0     * CIL library *:* CIL module *
 0002:000015b8       $chain$5$?SaveAdapterInfo@AsiBluLinkConfigAdapterInfo@@QEAAXPEAVDialogParameters@@_N@Z 00000001800085b8     * CIL library *:* CIL module *
 0002:000015d8       $chain$6$?SaveAdapterInfo@AsiBluLinkConfigAdapterInfo@@QEAAXPEAVDialogParameters@@_N@Z 00000001800085d8     * CIL library *:* CIL module *
 0002:000015e8       $chain$7$?SaveAdapterInfo@AsiBluLinkConfigAdapterInfo@@QEAAXPEAVDialogParameters@@_N@Z 00000001800085e8     * CIL library *:* CIL module *
 0002:000015f8       $unwind$__raise_securityfailure 00000001800085f8     * CIL library *:* CIL module *
 0002:000015f8       $unwind$__atonexitinit     00000001800085f8     * CIL library *:* CIL module *
 0002:000015f8       $unwind$pre_c_init         00000001800085f8     * CIL library *:* CIL module *
 0002:000015f8       $unwind$__GSHandlerCheckCommon 00000001800085f8     * CIL library *:* CIL module *
 0002:000015f8       $unwind$DllMain            00000001800085f8     * CIL library *:* CIL module *
 0002:000015f8       $unwind$?RebootDialogProc@@YA_JPEAUHWND__@@I_K_J@Z 00000001800085f8     * CIL library *:* CIL module *
 0002:000015f8       $unwind$??1DialogParameters@@QEAA@XZ 00000001800085f8     * CIL library *:* CIL module *
 0002:00001600       $unwind$?ShowControlPanel_RunDll@@YAXPEAUHWND__@@PEAUHINSTANCE__@@PEADH@Z 0000000180008600     * CIL library *:* CIL module *
 0002:00001614       $chain$1$?ShowControlPanel_RunDll@@YAXPEAUHWND__@@PEAUHINSTANCE__@@PEADH@Z 0000000180008614     * CIL library *:* CIL module *
 0002:00001628       $chain$2$?ShowControlPanel_RunDll@@YAXPEAUHWND__@@PEAUHINSTANCE__@@PEADH@Z 0000000180008628     * CIL library *:* CIL module *
 0002:00001638       $unwind$?RegisterControlPanelApplet_RunDll@@YAXPEAUHWND__@@PEAUHINSTANCE__@@PEADH@Z 0000000180008638     * CIL library *:* CIL module *
 0002:00001648       $chain$1$?RegisterControlPanelApplet_RunDll@@YAXPEAUHWND__@@PEAUHINSTANCE__@@PEADH@Z 0000000180008648     * CIL library *:* CIL module *
 0002:0000165c       $chain$2$?RegisterControlPanelApplet_RunDll@@YAXPEAUHWND__@@PEAUHINSTANCE__@@PEADH@Z 000000018000865c     * CIL library *:* CIL module *
 0002:0000166c       $unwind$?DllRegisterServer@@YAJXZ 000000018000866c     * CIL library *:* CIL module *
 0002:00001678       $chain$0$?DllRegisterServer@@YAJXZ 0000000180008678     * CIL library *:* CIL module *
 0002:0000168c       $chain$1$?DllRegisterServer@@YAJXZ 000000018000868c     * CIL library *:* CIL module *
 0002:000016a0       $chain$2$?DllRegisterServer@@YAJXZ 00000001800086a0     * CIL library *:* CIL module *
 0002:000016b0       $chain$3$?DllRegisterServer@@YAJXZ 00000001800086b0     * CIL library *:* CIL module *
 0002:000016c0       $unwind$?DllUnregisterServer@@YAJXZ 00000001800086c0     * CIL library *:* CIL module *
 0002:000016c8       $unwind$?ReplaceBackgroundColor@@YAXPEAUHWND__@@K@Z 00000001800086c8     * CIL library *:* CIL module *
 0002:000016e0       $unwind$?BluLinkChannelEditSubclassProc@@YA_JPEAUHWND__@@I_K_J11@Z 00000001800086e0     * CIL library *:* CIL module *
 0002:000016f4       $chain$0$?BluLinkChannelEditSubclassProc@@YA_JPEAUHWND__@@I_K_J11@Z 00000001800086f4     * CIL library *:* CIL module *
 0002:00001708       $chain$1$?BluLinkChannelEditSubclassProc@@YA_JPEAUHWND__@@I_K_J11@Z 0000000180008708     * CIL library *:* CIL module *
 0002:00001718       $unwind$swprintf           0000000180008718     * CIL library *:* CIL module *
 0002:00001718       $unwind$swprintf           0000000180008718     * CIL library *:* CIL module *
 0002:00001720       $unwind$_onexit$fin$0      0000000180008720     * CIL library *:* CIL module *
 0002:00001720       $unwind$__DllMainCRTStartup$filt$0 0000000180008720     * CIL library *:* CIL module *
 0002:00001720       $unwind$??1AsiBluLinkConfigAdapterInfo@@QEAA@XZ 0000000180008720     * CIL library *:* CIL module *
 0002:00001720       $unwind$__DllMainCRTStartup$fin$1 0000000180008720     * CIL library *:* CIL module *
 0002:00001720       $unwind$_IsNonwritableInCurrentImage$filt$0 0000000180008720     * CIL library *:* CIL module *
 0002:00001728       $chain$0$??1AsiBluLinkConfigAdapterInfo@@QEAA@XZ 0000000180008728     * CIL library *:* CIL module *
 0002:0000173c       $chain$2$??1AsiBluLinkConfigAdapterInfo@@QEAA@XZ 000000018000873c     * CIL library *:* CIL module *
 0002:00001754       $chain$3$??1AsiBluLinkConfigAdapterInfo@@QEAA@XZ 0000000180008754     * CIL library *:* CIL module *
 0002:00001764       $chain$4$??1AsiBluLinkConfigAdapterInfo@@QEAA@XZ 0000000180008764     * CIL library *:* CIL module *
 0002:00001774       $unwind$?KeyboardProc@KeyboardHook@@CA_JH_K_J@Z 0000000180008774     * CIL library *:* CIL module *
 0002:0000177c       $unwind$?CheckInitialSettings@DialogParameters@@QEAAXPEAUHWND__@@@Z 000000018000877c     * CIL library *:* CIL module *
 0002:00001788       $chain$1$?CheckInitialSettings@DialogParameters@@QEAAXPEAUHWND__@@@Z 0000000180008788     * CIL library *:* CIL module *
 0002:000017a0       $chain$2$?CheckInitialSettings@DialogParameters@@QEAAXPEAUHWND__@@@Z 00000001800087a0     * CIL library *:* CIL module *
 0002:000017b4       $chain$3$?CheckInitialSettings@DialogParameters@@QEAAXPEAUHWND__@@@Z 00000001800087b4     * CIL library *:* CIL module *
 0002:000017c4       $chain$4$?CheckInitialSettings@DialogParameters@@QEAAXPEAUHWND__@@@Z 00000001800087c4     * CIL library *:* CIL module *
 0002:000017d4       $unwind$?CreateGroupOfControls@DialogParameters@@QEAAPEAGPEAGHHKKK@Z 00000001800087d4     * CIL library *:* CIL module *
 0002:000017ec       $chain$0$?CreateGroupOfControls@DialogParameters@@QEAAPEAGPEAGHHKKK@Z 00000001800087ec     * CIL library *:* CIL module *
 0002:00001800       $chain$1$?CreateGroupOfControls@DialogParameters@@QEAAPEAGPEAGHHKKK@Z 0000000180008800     * CIL library *:* CIL module *
 0002:00001810       $unwind$?CustomizeDialog@DialogParameters@@QEAAPEAEPEAEH@Z 0000000180008810     * CIL library *:* CIL module *
 0002:0000182c       $unwind$?CheckTxConflicts@DialogParameters@@QEAAXPEAVBluLinkChannelControl@@@Z 000000018000882c     * CIL library *:* CIL module *
 0002:00001848       $unwind$?RunRebootDialog@DialogParameters@@QEAAHPEAUHWND__@@@Z 0000000180008848     * CIL library *:* CIL module *
 0002:0000185c       $unwind$?CheckSampleRateMismatch@DialogParameters@@QEAAHPEAUHWND__@@@Z 000000018000885c     * CIL library *:* CIL module *
 0002:0000186c       $chain$1$?CheckSampleRateMismatch@DialogParameters@@QEAAHPEAUHWND__@@@Z 000000018000886c     * CIL library *:* CIL module *
 0002:00001884       $chain$2$?CheckSampleRateMismatch@DialogParameters@@QEAAHPEAUHWND__@@@Z 0000000180008884     * CIL library *:* CIL module *
 0002:00001898       $chain$3$?CheckSampleRateMismatch@DialogParameters@@QEAAHPEAUHWND__@@@Z 0000000180008898     * CIL library *:* CIL module *
 0002:000018a8       $chain$4$?CheckSampleRateMismatch@DialogParameters@@QEAAHPEAUHWND__@@@Z 00000001800088a8     * CIL library *:* CIL module *
 0002:000018b8       $unwind$?GuiSamplerateChange@DialogParameters@@QEAAXPEAUHWND__@@H@Z 00000001800088b8     * CIL library *:* CIL module *
 0002:000018d4       $unwind$??0AsiScrollbar@@QEAA@PEAUHWND__@@HHH@Z 00000001800088d4     * CIL library *:* CIL module *
 0002:000018e4       $unwind$?HandleScrollMessage@AsiScrollbar@@QEAAXGG@Z 00000001800088e4     * CIL library *:* CIL module *
 0002:000018f4       $unwind$?InitControls@@YAXPEAUHWND__@@PEAVDialogParameters@@@Z 00000001800088f4     * CIL library *:* CIL module *
 0002:00001910       $chain$0$?InitControls@@YAXPEAUHWND__@@PEAVDialogParameters@@@Z 0000000180008910     * CIL library *:* CIL module *
 0002:00001924       $unwind$?CalculateMaxScroll@@YAHPEAUHWND__@@@Z 0000000180008924     * CIL library *:* CIL module *
 0002:00001934       $unwind$?SetChannelValue@@YAXPEAUHWND__@@PEAVBluLinkChannelControl@@PEAVDialogParameters@@_KH@Z 0000000180008934     * CIL library *:* CIL module *
 0002:00001934       $unwind$_DllMainCRTStartup 0000000180008934     * CIL library *:* CIL module *
 0002:00001944       $unwind$?EditControlMessage@@YA_JPEAUHWND__@@_K_JPEAVDialogParameters@@@Z 0000000180008944     * CIL library *:* CIL module *
 0002:0000195c       $unwind$?GetShutdownPrivilege@@YAXXZ 000000018000895c     * CIL library *:* CIL module *
 0002:0000196c       $unwind$?DialogProc@@YA_JPEAUHWND__@@I_K_J@Z 000000018000896c     * CIL library *:* CIL module *
 0002:00001988       $unwind$?SetControlToBold@@YAXPEAUHWND__@@H@Z 0000000180008988     * CIL library *:* CIL module *
 0002:000019a4       $unwind$?RunDialog@@YAXPEAUHWND__@@_N@Z 00000001800089a4     * CIL library *:* CIL module *
 0002:000019c4       $stateUnwindMap$?RunDialog@@YAXPEAUHWND__@@_N@Z 00000001800089c4     * CIL library *:* CIL module *
 0002:000019d4       $ip2state$?RunDialog@@YAXPEAUHWND__@@_N@Z 00000001800089d4     * CIL library *:* CIL module *
 0002:000019f8       $xdatasym                  00000001800089f8     MSVCRT:amdsecgs.obj
 0002:000019fc       $unwind$_CRT_INIT          00000001800089fc     MSVCRT:crtdll.obj
 0002:00001a18       $unwind$__DllMainCRTStartup 0000000180008a18     MSVCRT:crtdll.obj
 0002:00001a54       $unwind$__report_gsfailure 0000000180008a54     MSVCRT:gs_report.obj
 0002:00001a5c       $unwind$_IsNonwritableInCurrentImage 0000000180008a5c     MSVCRT:pesect.obj
 0002:00001a80       $unwind$_onexit            0000000180008a80     MSVCRT:atonexit.obj
 0002:00001aa0       $unwind$__security_init_cookie 0000000180008aa0     MSVCRT:gs_support.obj
 0002:00001aac       $unwind$_RTC_Terminate     0000000180008aac     MSVCRT:initsect.obj
 0002:00001aac       $unwind$_RTC_Initialize    0000000180008aac     MSVCRT:initsect.obj
 0002:00001ab8       $unwind$atexit             0000000180008ab8     MSVCRT:gshandler.obj
 0002:00001ab8       $unwind$__GSHandlerCheck   0000000180008ab8     MSVCRT:gshandler.obj
 0002:00001ac0       .edata                     0000000180008ac0     AsiBlCfg64.exp
 0002:00001ae8       rgpv                       0000000180008ae8     AsiBlCfg64.exp
 0002:00001af8       rgszName                   0000000180008af8     AsiBlCfg64.exp
 0002:00001b08       rgwOrd                     0000000180008b08     AsiBlCfg64.exp
 0002:00001b10       szName                     0000000180008b10     AsiBlCfg64.exp
 0002:00001b1f       $N00001                    0000000180008b1f     AsiBlCfg64.exp
 0002:00001b31       $N00002                    0000000180008b31     AsiBlCfg64.exp
 0002:00001b45       $N00003                    0000000180008b45     AsiBlCfg64.exp
 0002:00001b67       $N00004                    0000000180008b67     AsiBlCfg64.exp
 0002:00002010       .idata$6                   0000000180009010     Comctl32:COMCTL32.dll
 0002:00002086       .idata$6                   0000000180009086     Setupapi:SETUPAPI.dll
 0002:00002238       .idata$6                   0000000180009238     asihpi64:ASIHPI64.dll
 0002:000022b8       .idata$6                   00000001800092b8     kernel32:KERNEL32.dll
 0002:0000251c       .idata$6                   000000018000951c     user32:USER32.dll
 0002:0000258e       .idata$6                   000000018000958e     gdi32:GDI32.dll
 0002:00002664       .idata$6                   0000000180009664     advapi32:ADVAPI32.dll
 0002:000026c6       .idata$6                   00000001800096c6     MSVCRT:MSVCR120.dll
 0003:00000020       ClassesEntrySubList2       000000018000a020     * CIL library *:* CIL module *
 0003:000000e8       ControlPanelNamespaceRegList 000000018000a0e8     * CIL library *:* CIL module *
 0003:00000100       ClassesEntryList           000000018000a100     * CIL library *:* CIL module *
 0003:00000268       ClassesRegList             000000018000a268     * CIL library *:* CIL module *
 0003:00000280       ControlPanelNamespaceEntryList 000000018000a280     * CIL library *:* CIL module *
 0003:000002f8       PolicyRegList              000000018000a2f8     * CIL library *:* CIL module *
 0003:00000310       ClassesEntrySubList1       000000018000a310     * CIL library *:* CIL module *
 0003:00000390       PolicyEntryList            000000018000a390     * CIL library *:* CIL module *
 0003:00000430       originalDialogResource     000000018000a430     * CIL library *:* CIL module *
 0003:00000720       __proc_attached            000000018000a720     MSVCRT:crtdll.obj
 0003:00000730       GS_ExceptionRecord         000000018000a730     MSVCRT:gs_report.obj
 0003:000007d0       GS_ContextRecord           000000018000a7d0     MSVCRT:gs_report.obj
 0003:00000ca0       DebuggerWasPresent         000000018000aca0     MSVCRT:gs_report.obj
 0003:00000dc0       ?pScrollbar@?1??DialogProc@@YA_JPEAUHWND__@@I_K_J@Z@4PEAVAsiScrollbar@@EA 000000018000adc0     * CIL library *:* CIL module *
 0004:00000000       $pdata$?AddList@ControlPanelRegistration@@AEAA_NPEAUkey_path_entry@@PEAUreg_list_entry@@@Z 000000018000b000     * CIL library *:* CIL module *
 0004:0000000c       $pdata$0$?AddList@ControlPanelRegistration@@AEAA_NPEAUkey_path_entry@@PEAUreg_list_entry@@@Z 000000018000b00c     * CIL library *:* CIL module *
 0004:00000018       $pdata$1$?AddList@ControlPanelRegistration@@AEAA_NPEAUkey_path_entry@@PEAUreg_list_entry@@@Z 000000018000b018     * CIL library *:* CIL module *
 0004:00000024       $pdata$2$?AddList@ControlPanelRegistration@@AEAA_NPEAUkey_path_entry@@PEAUreg_list_entry@@@Z 000000018000b024     * CIL library *:* CIL module *
 0004:00000030       $pdata$?RemoveList@ControlPanelRegistration@@AEAA_NPEAUkey_path_entry@@PEAUreg_list_entry@@@Z 000000018000b030     * CIL library *:* CIL module *
 0004:0000003c       $pdata$0$?RemoveList@ControlPanelRegistration@@AEAA_NPEAUkey_path_entry@@PEAUreg_list_entry@@@Z 000000018000b03c     * CIL library *:* CIL module *
 0004:00000048       $pdata$1$?RemoveList@ControlPanelRegistration@@AEAA_NPEAUkey_path_entry@@PEAUreg_list_entry@@@Z 000000018000b048     * CIL library *:* CIL module *
 0004:00000054       $pdata$?FindValueName@ControlPanelRegistration@@AEAA_NPEAUHKEY__@@PEB_WPEA_WH@Z 000000018000b054     * CIL library *:* CIL module *
 0004:00000060       $pdata$?IsRegistered@ControlPanelRegistration@@QEAA?AW4CPRegState@@XZ 000000018000b060     * CIL library *:* CIL module *
 0004:0000006c       $pdata$?Register@ControlPanelRegistration@@QEAA_NXZ 000000018000b06c     * CIL library *:* CIL module *
 0004:00000078       $pdata$2$?Register@ControlPanelRegistration@@QEAA_NXZ 000000018000b078     * CIL library *:* CIL module *
 0004:00000084       $pdata$3$?Register@ControlPanelRegistration@@QEAA_NXZ 000000018000b084     * CIL library *:* CIL module *
 0004:00000090       $pdata$?UnRegister@ControlPanelRegistration@@QEAA_NXZ 000000018000b090     * CIL library *:* CIL module *
 0004:0000009c       $pdata$2$?UnRegister@ControlPanelRegistration@@QEAA_NXZ 000000018000b09c     * CIL library *:* CIL module *
 0004:000000a8       $pdata$3$?UnRegister@ControlPanelRegistration@@QEAA_NXZ 000000018000b0a8     * CIL library *:* CIL module *
 0004:000000b4       $pdata$?Show@ControlPanelRegistration@@QEAA_N_N@Z 000000018000b0b4     * CIL library *:* CIL module *
 0004:000000c0       $pdata$0$?Show@ControlPanelRegistration@@QEAA_N_N@Z 000000018000b0c0     * CIL library *:* CIL module *
 0004:000000cc       $pdata$1$?Show@ControlPanelRegistration@@QEAA_N_N@Z 000000018000b0cc     * CIL library *:* CIL module *
 0004:000000d8       $pdata$?SetChannel@BluLinkChannelControl@@QEAAXH@Z 000000018000b0d8     * CIL library *:* CIL module *
 0004:000000e4       $pdata$?SetChannelsPerDevice@DialogParameters@@QEAAXH@Z 000000018000b0e4     * CIL library *:* CIL module *
 0004:000000f0       $pdata$0$?SetChannelsPerDevice@DialogParameters@@QEAAXH@Z 000000018000b0f0     * CIL library *:* CIL module *
 0004:000000fc       $pdata$1$?SetChannelsPerDevice@DialogParameters@@QEAAXH@Z 000000018000b0fc     * CIL library *:* CIL module *
 0004:00000108       $pdata$?AllocateBlulinkControls@DialogParameters@@QEAAXXZ 000000018000b108     * CIL library *:* CIL module *
 0004:00000114       $pdata$0$?AllocateBlulinkControls@DialogParameters@@QEAAXXZ 000000018000b114     * CIL library *:* CIL module *
 0004:00000120       $pdata$2$?AllocateBlulinkControls@DialogParameters@@QEAAXXZ 000000018000b120     * CIL library *:* CIL module *
 0004:0000012c       $pdata$3$?AllocateBlulinkControls@DialogParameters@@QEAAXXZ 000000018000b12c     * CIL library *:* CIL module *
 0004:00000138       $pdata$4$?AllocateBlulinkControls@DialogParameters@@QEAAXXZ 000000018000b138     * CIL library *:* CIL module *
 0004:00000144       $pdata$5$?AllocateBlulinkControls@DialogParameters@@QEAAXXZ 000000018000b144     * CIL library *:* CIL module *
 0004:00000150       $pdata$?FoundAsiRegistryKey@AsiBluLinkConfigPerAdapterInfo@@QEAAHPEAVDialogParameters@@PEAUHKEY__@@@Z 000000018000b150     * CIL library *:* CIL module *
 0004:0000015c       $pdata$?GetChannelFromHpiControl@@YAHII@Z 000000018000b15c     * CIL library *:* CIL module *
 0004:00000168       $pdata$?InitChannels@AsiBluLinkConfigPerAdapterInfo@@QEAAXPEAVDialogParameters@@PEAX@Z 000000018000b168     * CIL library *:* CIL module *
 0004:00000174       $pdata$2$?InitChannels@AsiBluLinkConfigPerAdapterInfo@@QEAAXPEAVDialogParameters@@PEAX@Z 000000018000b174     * CIL library *:* CIL module *
 0004:00000180       $pdata$3$?InitChannels@AsiBluLinkConfigPerAdapterInfo@@QEAAXPEAVDialogParameters@@PEAX@Z 000000018000b180     * CIL library *:* CIL module *
 0004:0000018c       $pdata$?SaveChannelToHpiControl@@YAXIIH@Z 000000018000b18c     * CIL library *:* CIL module *
 0004:00000198       $pdata$?SaveChannels@AsiBluLinkConfigPerAdapterInfo@@QEAAXPEAVDialogParameters@@PEAX@Z 000000018000b198     * CIL library *:* CIL module *
 0004:000001a4       $pdata$0$?SaveChannels@AsiBluLinkConfigPerAdapterInfo@@QEAAXPEAVDialogParameters@@PEAX@Z 000000018000b1a4     * CIL library *:* CIL module *
 0004:000001b0       $pdata$6$?SaveChannels@AsiBluLinkConfigPerAdapterInfo@@QEAAXPEAVDialogParameters@@PEAX@Z 000000018000b1b0     * CIL library *:* CIL module *
 0004:000001bc       $pdata$7$?SaveChannels@AsiBluLinkConfigPerAdapterInfo@@QEAAXPEAVDialogParameters@@PEAX@Z 000000018000b1bc     * CIL library *:* CIL module *
 0004:000001c8       $pdata$8$?SaveChannels@AsiBluLinkConfigPerAdapterInfo@@QEAAXPEAVDialogParameters@@PEAX@Z 000000018000b1c8     * CIL library *:* CIL module *
 0004:000001d4       $pdata$?FoundAsiRegistryKey@AsiBluLinkConfigAdapterInfo@@AEAAHPEAVDialogParameters@@PEAUHKEY__@@@Z 000000018000b1d4     * CIL library *:* CIL module *
 0004:000001e0       $pdata$?InitChannelsPerDevice@AsiBluLinkConfigAdapterInfo@@AEAAXPEAVDialogParameters@@PEAUHWND__@@@Z 000000018000b1e0     * CIL library *:* CIL module *
 0004:000001ec       $pdata$2$?InitChannelsPerDevice@AsiBluLinkConfigAdapterInfo@@AEAAXPEAVDialogParameters@@PEAUHWND__@@@Z 000000018000b1ec     * CIL library *:* CIL module *
 0004:000001f8       $pdata$3$?InitChannelsPerDevice@AsiBluLinkConfigAdapterInfo@@AEAAXPEAVDialogParameters@@PEAUHWND__@@@Z 000000018000b1f8     * CIL library *:* CIL module *
 0004:00000204       $pdata$4$?InitChannelsPerDevice@AsiBluLinkConfigAdapterInfo@@AEAAXPEAVDialogParameters@@PEAUHWND__@@@Z 000000018000b204     * CIL library *:* CIL module *
 0004:00000210       $pdata$5$?InitChannelsPerDevice@AsiBluLinkConfigAdapterInfo@@AEAAXPEAVDialogParameters@@PEAUHWND__@@@Z 000000018000b210     * CIL library *:* CIL module *
 0004:0000021c       $pdata$6$?InitChannelsPerDevice@AsiBluLinkConfigAdapterInfo@@AEAAXPEAVDialogParameters@@PEAUHWND__@@@Z 000000018000b21c     * CIL library *:* CIL module *
 0004:00000228       $pdata$?InitAdapterInfo@AsiBluLinkConfigAdapterInfo@@QEAAHPEAVDialogParameters@@PEAUHWND__@@_N@Z 000000018000b228     * CIL library *:* CIL module *
 0004:00000234       $pdata$?SaveAdapterInfo@AsiBluLinkConfigAdapterInfo@@QEAAXPEAVDialogParameters@@_N@Z 000000018000b234     * CIL library *:* CIL module *
 0004:00000240       $pdata$1$?SaveAdapterInfo@AsiBluLinkConfigAdapterInfo@@QEAAXPEAVDialogParameters@@_N@Z 000000018000b240     * CIL library *:* CIL module *
 0004:0000024c       $pdata$5$?SaveAdapterInfo@AsiBluLinkConfigAdapterInfo@@QEAAXPEAVDialogParameters@@_N@Z 000000018000b24c     * CIL library *:* CIL module *
 0004:00000258       $pdata$6$?SaveAdapterInfo@AsiBluLinkConfigAdapterInfo@@QEAAXPEAVDialogParameters@@_N@Z 000000018000b258     * CIL library *:* CIL module *
 0004:00000264       $pdata$7$?SaveAdapterInfo@AsiBluLinkConfigAdapterInfo@@QEAAXPEAVDialogParameters@@_N@Z 000000018000b264     * CIL library *:* CIL module *
 0004:00000270       $pdata$DllMain             000000018000b270     * CIL library *:* CIL module *
 0004:0000027c       $pdata$?ShowControlPanel_RunDll@@YAXPEAUHWND__@@PEAUHINSTANCE__@@PEADH@Z 000000018000b27c     * CIL library *:* CIL module *
 0004:00000288       $pdata$1$?ShowControlPanel_RunDll@@YAXPEAUHWND__@@PEAUHINSTANCE__@@PEADH@Z 000000018000b288     * CIL library *:* CIL module *
 0004:00000294       $pdata$2$?ShowControlPanel_RunDll@@YAXPEAUHWND__@@PEAUHINSTANCE__@@PEADH@Z 000000018000b294     * CIL library *:* CIL module *
 0004:000002a0       $pdata$?RegisterControlPanelApplet_RunDll@@YAXPEAUHWND__@@PEAUHINSTANCE__@@PEADH@Z 000000018000b2a0     * CIL library *:* CIL module *
 0004:000002ac       $pdata$1$?RegisterControlPanelApplet_RunDll@@YAXPEAUHWND__@@PEAUHINSTANCE__@@PEADH@Z 000000018000b2ac     * CIL library *:* CIL module *
 0004:000002b8       $pdata$2$?RegisterControlPanelApplet_RunDll@@YAXPEAUHWND__@@PEAUHINSTANCE__@@PEADH@Z 000000018000b2b8     * CIL library *:* CIL module *
 0004:000002c4       $pdata$?DllRegisterServer@@YAJXZ 000000018000b2c4     * CIL library *:* CIL module *
 0004:000002d0       $pdata$0$?DllRegisterServer@@YAJXZ 000000018000b2d0     * CIL library *:* CIL module *
 0004:000002dc       $pdata$1$?DllRegisterServer@@YAJXZ 000000018000b2dc     * CIL library *:* CIL module *
 0004:000002e8       $pdata$2$?DllRegisterServer@@YAJXZ 000000018000b2e8     * CIL library *:* CIL module *
 0004:000002f4       $pdata$3$?DllRegisterServer@@YAJXZ 000000018000b2f4     * CIL library *:* CIL module *
 0004:00000300       $pdata$?DllUnregisterServer@@YAJXZ 000000018000b300     * CIL library *:* CIL module *
 0004:0000030c       $pdata$?SetConflict@BluLinkChannelControl@@QEAAXPEAV1@@Z 000000018000b30c     * CIL library *:* CIL module *
 0004:00000318       $pdata$?ReplaceBackgroundColor@@YAXPEAUHWND__@@K@Z 000000018000b318     * CIL library *:* CIL module *
 0004:00000324       $pdata$?BluLinkChannelEditSubclassProc@@YA_JPEAUHWND__@@I_K_J11@Z 000000018000b324     * CIL library *:* CIL module *
 0004:00000330       $pdata$0$?BluLinkChannelEditSubclassProc@@YA_JPEAUHWND__@@I_K_J11@Z 000000018000b330     * CIL library *:* CIL module *
 0004:0000033c       $pdata$1$?BluLinkChannelEditSubclassProc@@YA_JPEAUHWND__@@I_K_J11@Z 000000018000b33c     * CIL library *:* CIL module *
 0004:00000348       $pdata$swprintf            000000018000b348     * CIL library *:* CIL module *
 0004:00000348       $pdata$swprintf            000000018000b348     * CIL library *:* CIL module *
 0004:00000354       $pdata$??1DialogParameters@@QEAA@XZ 000000018000b354     * CIL library *:* CIL module *
 0004:00000360       $pdata$??1AsiBluLinkConfigAdapterInfo@@QEAA@XZ 000000018000b360     * CIL library *:* CIL module *
 0004:0000036c       $pdata$0$??1AsiBluLinkConfigAdapterInfo@@QEAA@XZ 000000018000b36c     * CIL library *:* CIL module *
 0004:00000378       $pdata$2$??1AsiBluLinkConfigAdapterInfo@@QEAA@XZ 000000018000b378     * CIL library *:* CIL module *
 0004:00000384       $pdata$3$??1AsiBluLinkConfigAdapterInfo@@QEAA@XZ 000000018000b384     * CIL library *:* CIL module *
 0004:00000390       $pdata$4$??1AsiBluLinkConfigAdapterInfo@@QEAA@XZ 000000018000b390     * CIL library *:* CIL module *
 0004:0000039c       $pdata$?KeyboardProc@KeyboardHook@@CA_JH_K_J@Z 000000018000b39c     * CIL library *:* CIL module *
 0004:000003a8       $pdata$?CheckInitialSettings@DialogParameters@@QEAAXPEAUHWND__@@@Z 000000018000b3a8     * CIL library *:* CIL module *
 0004:000003b4       $pdata$1$?CheckInitialSettings@DialogParameters@@QEAAXPEAUHWND__@@@Z 000000018000b3b4     * CIL library *:* CIL module *
 0004:000003c0       $pdata$2$?CheckInitialSettings@DialogParameters@@QEAAXPEAUHWND__@@@Z 000000018000b3c0     * CIL library *:* CIL module *
 0004:000003cc       $pdata$3$?CheckInitialSettings@DialogParameters@@QEAAXPEAUHWND__@@@Z 000000018000b3cc     * CIL library *:* CIL module *
 0004:000003d8       $pdata$4$?CheckInitialSettings@DialogParameters@@QEAAXPEAUHWND__@@@Z 000000018000b3d8     * CIL library *:* CIL module *
 0004:000003e4       $pdata$?CreateGroupOfControls@DialogParameters@@QEAAPEAGPEAGHHKKK@Z 000000018000b3e4     * CIL library *:* CIL module *
 0004:000003f0       $pdata$0$?CreateGroupOfControls@DialogParameters@@QEAAPEAGPEAGHHKKK@Z 000000018000b3f0     * CIL library *:* CIL module *
 0004:000003fc       $pdata$1$?CreateGroupOfControls@DialogParameters@@QEAAPEAGPEAGHHKKK@Z 000000018000b3fc     * CIL library *:* CIL module *
 0004:00000408       $pdata$?CustomizeDialog@DialogParameters@@QEAAPEAEPEAEH@Z 000000018000b408     * CIL library *:* CIL module *
 0004:00000414       $pdata$?CheckTxConflicts@DialogParameters@@QEAAXPEAVBluLinkChannelControl@@@Z 000000018000b414     * CIL library *:* CIL module *
 0004:00000420       $pdata$?RunRebootDialog@DialogParameters@@QEAAHPEAUHWND__@@@Z 000000018000b420     * CIL library *:* CIL module *
 0004:0000042c       $pdata$?CheckSampleRateMismatch@DialogParameters@@QEAAHPEAUHWND__@@@Z 000000018000b42c     * CIL library *:* CIL module *
 0004:00000438       $pdata$1$?CheckSampleRateMismatch@DialogParameters@@QEAAHPEAUHWND__@@@Z 000000018000b438     * CIL library *:* CIL module *
 0004:00000444       $pdata$2$?CheckSampleRateMismatch@DialogParameters@@QEAAHPEAUHWND__@@@Z 000000018000b444     * CIL library *:* CIL module *
 0004:00000450       $pdata$3$?CheckSampleRateMismatch@DialogParameters@@QEAAHPEAUHWND__@@@Z 000000018000b450     * CIL library *:* CIL module *
 0004:0000045c       $pdata$4$?CheckSampleRateMismatch@DialogParameters@@QEAAHPEAUHWND__@@@Z 000000018000b45c     * CIL library *:* CIL module *
 0004:00000468       $pdata$?GuiSamplerateChange@DialogParameters@@QEAAXPEAUHWND__@@H@Z 000000018000b468     * CIL library *:* CIL module *
 0004:00000474       $pdata$??0AsiScrollbar@@QEAA@PEAUHWND__@@HHH@Z 000000018000b474     * CIL library *:* CIL module *
 0004:00000480       $pdata$?HandleScrollMessage@AsiScrollbar@@QEAAXGG@Z 000000018000b480     * CIL library *:* CIL module *
 0004:0000048c       $pdata$?InitControls@@YAXPEAUHWND__@@PEAVDialogParameters@@@Z 000000018000b48c     * CIL library *:* CIL module *
 0004:00000498       $pdata$0$?InitControls@@YAXPEAUHWND__@@PEAVDialogParameters@@@Z 000000018000b498     * CIL library *:* CIL module *
 0004:000004a4       $pdata$?CalculateMaxScroll@@YAHPEAUHWND__@@@Z 000000018000b4a4     * CIL library *:* CIL module *
 0004:000004b0       $pdata$?SetChannelValue@@YAXPEAUHWND__@@PEAVBluLinkChannelControl@@PEAVDialogParameters@@_KH@Z 000000018000b4b0     * CIL library *:* CIL module *
 0004:000004bc       $pdata$?EditControlMessage@@YA_JPEAUHWND__@@_K_JPEAVDialogParameters@@@Z 000000018000b4bc     * CIL library *:* CIL module *
 0004:000004c8       $pdata$?GetShutdownPrivilege@@YAXXZ 000000018000b4c8     * CIL library *:* CIL module *
 0004:000004d4       $pdata$?DialogProc@@YA_JPEAUHWND__@@I_K_J@Z 000000018000b4d4     * CIL library *:* CIL module *
 0004:000004e0       $pdata$?SetControlToBold@@YAXPEAUHWND__@@H@Z 000000018000b4e0     * CIL library *:* CIL module *
 0004:000004ec       $pdata$?RebootDialogProc@@YA_JPEAUHWND__@@I_K_J@Z 000000018000b4ec     * CIL library *:* CIL module *
 0004:000004f8       $pdata$?RunDialog@@YAXPEAUHWND__@@_N@Z 000000018000b4f8     * CIL library *:* CIL module *
 0004:00000510       $pdata$pre_c_init          000000018000b510     MSVCRT:crtdll.obj
 0004:0000051c       $pdata$_CRT_INIT           000000018000b51c     MSVCRT:crtdll.obj
 0004:00000528       $pdata$_DllMainCRTStartup  000000018000b528     MSVCRT:crtdll.obj
 0004:00000534       $pdata$__DllMainCRTStartup 000000018000b534     MSVCRT:crtdll.obj
 0004:00000540       $pdata$__raise_securityfailure 000000018000b540     MSVCRT:gs_report.obj
 0004:0000054c       $pdata$__report_gsfailure  000000018000b54c     MSVCRT:gs_report.obj
 0004:00000558       $pdata$_IsNonwritableInCurrentImage 000000018000b558     MSVCRT:pesect.obj
 0004:00000564       $pdata$__atonexitinit      000000018000b564     MSVCRT:atonexit.obj
 0004:00000570       $pdata$_onexit             000000018000b570     MSVCRT:atonexit.obj
 0004:0000057c       $pdata$atexit              000000018000b57c     MSVCRT:atonexit.obj
 0004:00000588       $pdata$__security_init_cookie 000000018000b588     MSVCRT:gs_support.obj
 0004:00000594       $pdata$_RTC_Initialize     000000018000b594     MSVCRT:initsect.obj
 0004:000005a0       $pdata$_RTC_Terminate      000000018000b5a0     MSVCRT:initsect.obj
 0004:000005ac       $pdata$__GSHandlerCheck    000000018000b5ac     MSVCRT:gshandler.obj
 0004:000005b8       $pdata$__GSHandlerCheckCommon 000000018000b5b8     MSVCRT:gshandler.obj
 0004:000005c4       $pdata$__DllMainCRTStartup$filt$0 000000018000b5c4     MSVCRT:crtdll.obj
 0004:000005d0       $pdata$__DllMainCRTStartup$fin$1 000000018000b5d0     MSVCRT:crtdll.obj
 0004:000005dc       $pdata$_IsNonwritableInCurrentImage$filt$0 000000018000b5dc     MSVCRT:pesect.obj
 0004:000005e8       $pdata$_onexit$fin$0       000000018000b5e8     MSVCRT:atonexit.obj
 0005:000002d0       $R000000                   000000018000c2d0     BluLinkCfg.res
 0005:00000f78       $R000CA8                   000000018000cf78     BluLinkCfg.res
 0005:00000f90       $R000CC0                   000000018000cf90     BluLinkCfg.res
 0005:00000fe0       $R000D10                   000000018000cfe0     BluLinkCfg.res
 0005:00000ff0       $R000D20                   000000018000cff0     BluLinkCfg.res
 0005:00001108       $R000E38                   000000018000d108     BluLinkCfg.res
 0005:00001478       $R0011A8                   000000018000d478     BluLinkCfg.res
 0005:0002c920       $R02C650                   0000000180038920     BluLinkCfg.res
 0005:0002cc78       $R02C9A8                   0000000180038c78     BluLinkCfg.res
 0005:0002cce0       $R02CA10                   0000000180038ce0     BluLinkCfg.res
